Component: Arm Compiler for Embedded 6.21 Tool: armlink [5ec1fa00]

==============================================================================

Section Cross References

    main.o(.text.fputc) refers to main.o(.text.DL_UART_isBusy) for DL_UART_isBusy
    main.o(.text.fputc) refers to main.o(.text.DL_UART_transmitData) for DL_UART_transmitData
    main.o(.ARM.exidx.text.fputc) refers to main.o(.text.fputc) for [Anonymous Symbol]
    main.o(.ARM.exidx.text.DL_UART_isBusy) refers to main.o(.text.DL_UART_isBusy) for [Anonymous Symbol]
    main.o(.ARM.exidx.text.DL_UART_transmitData) refers to main.o(.text.DL_UART_transmitData) for [Anonymous Symbol]
    main.o(.text.CalculateNormalizedValue) refers to idiv_div0.o(.text) for __aeabi_idiv
    main.o(.text.CalculateNormalizedValue) refers to main.o(.bss.CalculateNormalizedValue.last_value) for [Anonymous Symbol]
    main.o(.ARM.exidx.text.CalculateNormalizedValue) refers to main.o(.text.CalculateNormalizedValue) for [Anonymous Symbol]
    main.o(.text.main) refers to ti_msp_dl_config.o(.text.SYSCFG_DL_init) for SYSCFG_DL_init
    main.o(.text.main) refers to main.o(.text.DL_DMA_setSrcAddr) for DL_DMA_setSrcAddr
    main.o(.text.main) refers to main.o(.text.DL_DMA_setDestAddr) for DL_DMA_setDestAddr
    main.o(.text.main) refers to main.o(.text.DL_DMA_enableChannel) for DL_DMA_enableChannel
    main.o(.text.main) refers to main.o(.text.DL_ADC12_startConversion) for DL_ADC12_startConversion
    main.o(.text.main) refers to no_mcu_ganv_grayscale_sensor.o(.text.No_MCU_Ganv_Sensor_Init) for No_MCU_Ganv_Sensor_Init
    main.o(.text.main) refers to printfa.o(i.__0printf) for printf
    main.o(.text.main) refers to main.o(.text.__NVIC_EnableIRQ) for __NVIC_EnableIRQ
    main.o(.text.main) refers to delay.o(.text.Tick_delay) for Tick_delay
    main.o(.text.main) refers to main.o(.text.DL_Timer_startCounter) for DL_Timer_startCounter
    main.o(.text.main) refers to no_mcu_ganv_grayscale_sensor.o(.text.No_Mcu_Ganv_Sensor_Task_Without_tick) for No_Mcu_Ganv_Sensor_Task_Without_tick
    main.o(.text.main) refers to no_mcu_ganv_grayscale_sensor.o(.text.Get_Normalize_For_User) for Get_Normalize_For_User
    main.o(.text.main) refers to no_mcu_ganv_grayscale_sensor.o(.text.Get_Digtal_For_User) for Get_Digtal_For_User
    main.o(.text.main) refers to main.o(.text.CalculateNormalizedValue) for CalculateNormalizedValue
    main.o(.text.main) refers to l298n.o(.text.Motor_Control) for Motor_Control
    main.o(.text.main) refers to adc.o(.bss.ADC_VALUE) for ADC_VALUE
    main.o(.text.main) refers to main.o(.bss.sensor) for sensor
    main.o(.text.main) refers to main.o(.data.white) for white
    main.o(.text.main) refers to main.o(.data.black) for black
    main.o(.text.main) refers to main.o(.rodata.str1.1) for [Anonymous Symbol]
    main.o(.text.main) refers to key.o(.bss.key_start_pressed) for key_start_pressed
    main.o(.text.main) refers to main.o(.bss.Normal) for Normal
    main.o(.text.main) refers to main.o(.bss.Digtal) for Digtal
    main.o(.text.main) refers to pid.o(.bss.result_angle) for result_angle
    main.o(.ARM.exidx.text.main) refers to main.o(.text.main) for [Anonymous Symbol]
    main.o(.ARM.exidx.text.DL_DMA_setSrcAddr) refers to main.o(.text.DL_DMA_setSrcAddr) for [Anonymous Symbol]
    main.o(.ARM.exidx.text.DL_DMA_setDestAddr) refers to main.o(.text.DL_DMA_setDestAddr) for [Anonymous Symbol]
    main.o(.ARM.exidx.text.DL_DMA_enableChannel) refers to main.o(.text.DL_DMA_enableChannel) for [Anonymous Symbol]
    main.o(.ARM.exidx.text.DL_ADC12_startConversion) refers to main.o(.text.DL_ADC12_startConversion) for [Anonymous Symbol]
    main.o(.ARM.exidx.text.__NVIC_EnableIRQ) refers to main.o(.text.__NVIC_EnableIRQ) for [Anonymous Symbol]
    main.o(.ARM.exidx.text.DL_Timer_startCounter) refers to main.o(.text.DL_Timer_startCounter) for [Anonymous Symbol]
    startup_mspm0l130x_uvision.o(RESET) refers to startup_mspm0l130x_uvision.o(STACK) for __initial_sp
    startup_mspm0l130x_uvision.o(RESET) refers to startup_mspm0l130x_uvision.o(.text) for Reset_Handler
    startup_mspm0l130x_uvision.o(RESET) refers to delay.o(.text.SysTick_Handler) for SysTick_Handler
    startup_mspm0l130x_uvision.o(RESET) refers to key.o(.text.GROUP1_IRQHandler) for GROUP1_IRQHandler
    startup_mspm0l130x_uvision.o(RESET) refers to l298n.o(.text.TIMG0_IRQHandler) for TIMG0_IRQHandler
    startup_mspm0l130x_uvision.o(.text) refers to entry.o(.ARM.Collect$$$$00000000) for __main
    ti_msp_dl_config.o(.text.SYSCFG_DL_init) refers to ti_msp_dl_config.o(.text.SYSCFG_DL_initPower) for SYSCFG_DL_initPower
    ti_msp_dl_config.o(.text.SYSCFG_DL_init) refers to ti_msp_dl_config.o(.text.SYSCFG_DL_GPIO_init) for SYSCFG_DL_GPIO_init
    ti_msp_dl_config.o(.text.SYSCFG_DL_init) refers to ti_msp_dl_config.o(.text.SYSCFG_DL_SYSCTL_init) for SYSCFG_DL_SYSCTL_init
    ti_msp_dl_config.o(.text.SYSCFG_DL_init) refers to ti_msp_dl_config.o(.text.SYSCFG_DL_TIMER_0_init) for SYSCFG_DL_TIMER_0_init
    ti_msp_dl_config.o(.text.SYSCFG_DL_init) refers to ti_msp_dl_config.o(.text.SYSCFG_DL_UART_0_init) for SYSCFG_DL_UART_0_init
    ti_msp_dl_config.o(.text.SYSCFG_DL_init) refers to ti_msp_dl_config.o(.text.SYSCFG_DL_ADC_VOLTAGE_init) for SYSCFG_DL_ADC_VOLTAGE_init
    ti_msp_dl_config.o(.text.SYSCFG_DL_init) refers to ti_msp_dl_config.o(.text.SYSCFG_DL_DMA_init) for SYSCFG_DL_DMA_init
    ti_msp_dl_config.o(.text.SYSCFG_DL_init) refers to ti_msp_dl_config.o(.text.SYSCFG_DL_SYSTICK_init) for SYSCFG_DL_SYSTICK_init
    ti_msp_dl_config.o(.ARM.exidx.text.SYSCFG_DL_init) refers to ti_msp_dl_config.o(.text.SYSCFG_DL_init) for [Anonymous Symbol]
    ti_msp_dl_config.o(.text.SYSCFG_DL_initPower) refers to ti_msp_dl_config.o(.text.DL_GPIO_reset) for DL_GPIO_reset
    ti_msp_dl_config.o(.text.SYSCFG_DL_initPower) refers to ti_msp_dl_config.o(.text.DL_Timer_reset) for DL_Timer_reset
    ti_msp_dl_config.o(.text.SYSCFG_DL_initPower) refers to ti_msp_dl_config.o(.text.DL_UART_reset) for DL_UART_reset
    ti_msp_dl_config.o(.text.SYSCFG_DL_initPower) refers to ti_msp_dl_config.o(.text.DL_ADC12_reset) for DL_ADC12_reset
    ti_msp_dl_config.o(.text.SYSCFG_DL_initPower) refers to ti_msp_dl_config.o(.text.DL_GPIO_enablePower) for DL_GPIO_enablePower
    ti_msp_dl_config.o(.text.SYSCFG_DL_initPower) refers to ti_msp_dl_config.o(.text.DL_Timer_enablePower) for DL_Timer_enablePower
    ti_msp_dl_config.o(.text.SYSCFG_DL_initPower) refers to ti_msp_dl_config.o(.text.DL_UART_enablePower) for DL_UART_enablePower
    ti_msp_dl_config.o(.text.SYSCFG_DL_initPower) refers to ti_msp_dl_config.o(.text.DL_ADC12_enablePower) for DL_ADC12_enablePower
    ti_msp_dl_config.o(.text.SYSCFG_DL_initPower) refers to dl_common.o(.text.DL_Common_delayCycles) for DL_Common_delayCycles
    ti_msp_dl_config.o(.ARM.exidx.text.SYSCFG_DL_initPower) refers to ti_msp_dl_config.o(.text.SYSCFG_DL_initPower) for [Anonymous Symbol]
    ti_msp_dl_config.o(.text.SYSCFG_DL_GPIO_init) refers to ti_msp_dl_config.o(.text.DL_GPIO_initPeripheralOutputFunction) for DL_GPIO_initPeripheralOutputFunction
    ti_msp_dl_config.o(.text.SYSCFG_DL_GPIO_init) refers to ti_msp_dl_config.o(.text.DL_GPIO_initPeripheralInputFunction) for DL_GPIO_initPeripheralInputFunction
    ti_msp_dl_config.o(.text.SYSCFG_DL_GPIO_init) refers to ti_msp_dl_config.o(.text.DL_GPIO_initDigitalOutput) for DL_GPIO_initDigitalOutput
    ti_msp_dl_config.o(.text.SYSCFG_DL_GPIO_init) refers to ti_msp_dl_config.o(.text.DL_GPIO_initDigitalInputFeatures) for DL_GPIO_initDigitalInputFeatures
    ti_msp_dl_config.o(.text.SYSCFG_DL_GPIO_init) refers to ti_msp_dl_config.o(.text.DL_GPIO_clearPins) for DL_GPIO_clearPins
    ti_msp_dl_config.o(.text.SYSCFG_DL_GPIO_init) refers to ti_msp_dl_config.o(.text.DL_GPIO_enableOutput) for DL_GPIO_enableOutput
    ti_msp_dl_config.o(.text.SYSCFG_DL_GPIO_init) refers to ti_msp_dl_config.o(.text.DL_GPIO_setUpperPinsPolarity) for DL_GPIO_setUpperPinsPolarity
    ti_msp_dl_config.o(.text.SYSCFG_DL_GPIO_init) refers to ti_msp_dl_config.o(.text.DL_GPIO_clearInterruptStatus) for DL_GPIO_clearInterruptStatus
    ti_msp_dl_config.o(.text.SYSCFG_DL_GPIO_init) refers to ti_msp_dl_config.o(.text.DL_GPIO_enableInterrupt) for DL_GPIO_enableInterrupt
    ti_msp_dl_config.o(.ARM.exidx.text.SYSCFG_DL_GPIO_init) refers to ti_msp_dl_config.o(.text.SYSCFG_DL_GPIO_init) for [Anonymous Symbol]
    ti_msp_dl_config.o(.text.SYSCFG_DL_SYSCTL_init) refers to ti_msp_dl_config.o(.text.DL_SYSCTL_setBORThreshold) for DL_SYSCTL_setBORThreshold
    ti_msp_dl_config.o(.text.SYSCFG_DL_SYSCTL_init) refers to ti_msp_dl_config.o(.text.DL_SYSCTL_setSYSOSCFreq) for DL_SYSCTL_setSYSOSCFreq
    ti_msp_dl_config.o(.text.SYSCFG_DL_SYSCTL_init) refers to ti_msp_dl_config.o(.text.DL_SYSCTL_enableMFPCLK) for DL_SYSCTL_enableMFPCLK
    ti_msp_dl_config.o(.text.SYSCFG_DL_SYSCTL_init) refers to ti_msp_dl_config.o(.text.__NVIC_SetPriority) for __NVIC_SetPriority
    ti_msp_dl_config.o(.ARM.exidx.text.SYSCFG_DL_SYSCTL_init) refers to ti_msp_dl_config.o(.text.SYSCFG_DL_SYSCTL_init) for [Anonymous Symbol]
    ti_msp_dl_config.o(.text.SYSCFG_DL_TIMER_0_init) refers to dl_timer.o(.text.DL_Timer_setClockConfig) for DL_Timer_setClockConfig
    ti_msp_dl_config.o(.text.SYSCFG_DL_TIMER_0_init) refers to dl_timer.o(.text.DL_Timer_initTimerMode) for DL_Timer_initTimerMode
    ti_msp_dl_config.o(.text.SYSCFG_DL_TIMER_0_init) refers to ti_msp_dl_config.o(.text.DL_Timer_enableInterrupt) for DL_Timer_enableInterrupt
    ti_msp_dl_config.o(.text.SYSCFG_DL_TIMER_0_init) refers to ti_msp_dl_config.o(.text.__NVIC_SetPriority) for __NVIC_SetPriority
    ti_msp_dl_config.o(.text.SYSCFG_DL_TIMER_0_init) refers to ti_msp_dl_config.o(.text.DL_Timer_enableClock) for DL_Timer_enableClock
    ti_msp_dl_config.o(.text.SYSCFG_DL_TIMER_0_init) refers to ti_msp_dl_config.o(.rodata.gTIMER_0ClockConfig) for [Anonymous Symbol]
    ti_msp_dl_config.o(.text.SYSCFG_DL_TIMER_0_init) refers to ti_msp_dl_config.o(.rodata.gTIMER_0TimerConfig) for [Anonymous Symbol]
    ti_msp_dl_config.o(.ARM.exidx.text.SYSCFG_DL_TIMER_0_init) refers to ti_msp_dl_config.o(.text.SYSCFG_DL_TIMER_0_init) for [Anonymous Symbol]
    ti_msp_dl_config.o(.text.SYSCFG_DL_UART_0_init) refers to dl_uart.o(.text.DL_UART_setClockConfig) for DL_UART_setClockConfig
    ti_msp_dl_config.o(.text.SYSCFG_DL_UART_0_init) refers to dl_uart.o(.text.DL_UART_init) for DL_UART_init
    ti_msp_dl_config.o(.text.SYSCFG_DL_UART_0_init) refers to ti_msp_dl_config.o(.text.DL_UART_setOversampling) for DL_UART_setOversampling
    ti_msp_dl_config.o(.text.SYSCFG_DL_UART_0_init) refers to ti_msp_dl_config.o(.text.DL_UART_setBaudRateDivisor) for DL_UART_setBaudRateDivisor
    ti_msp_dl_config.o(.text.SYSCFG_DL_UART_0_init) refers to ti_msp_dl_config.o(.text.DL_UART_enable) for DL_UART_enable
    ti_msp_dl_config.o(.text.SYSCFG_DL_UART_0_init) refers to ti_msp_dl_config.o(.rodata.gUART_0ClockConfig) for [Anonymous Symbol]
    ti_msp_dl_config.o(.text.SYSCFG_DL_UART_0_init) refers to ti_msp_dl_config.o(.rodata.gUART_0Config) for [Anonymous Symbol]
    ti_msp_dl_config.o(.ARM.exidx.text.SYSCFG_DL_UART_0_init) refers to ti_msp_dl_config.o(.text.SYSCFG_DL_UART_0_init) for [Anonymous Symbol]
    ti_msp_dl_config.o(.text.SYSCFG_DL_ADC_VOLTAGE_init) refers to dl_adc12.o(.text.DL_ADC12_setClockConfig) for DL_ADC12_setClockConfig
    ti_msp_dl_config.o(.text.SYSCFG_DL_ADC_VOLTAGE_init) refers to ti_msp_dl_config.o(.text.DL_ADC12_initSingleSample) for DL_ADC12_initSingleSample
    ti_msp_dl_config.o(.text.SYSCFG_DL_ADC_VOLTAGE_init) refers to ti_msp_dl_config.o(.text.DL_ADC12_configConversionMem) for DL_ADC12_configConversionMem
    ti_msp_dl_config.o(.text.SYSCFG_DL_ADC_VOLTAGE_init) refers to ti_msp_dl_config.o(.text.DL_ADC12_setSampleTime0) for DL_ADC12_setSampleTime0
    ti_msp_dl_config.o(.text.SYSCFG_DL_ADC_VOLTAGE_init) refers to ti_msp_dl_config.o(.text.DL_ADC12_enableDMA) for DL_ADC12_enableDMA
    ti_msp_dl_config.o(.text.SYSCFG_DL_ADC_VOLTAGE_init) refers to ti_msp_dl_config.o(.text.DL_ADC12_setDMASamplesCnt) for DL_ADC12_setDMASamplesCnt
    ti_msp_dl_config.o(.text.SYSCFG_DL_ADC_VOLTAGE_init) refers to ti_msp_dl_config.o(.text.DL_ADC12_enableDMATrigger) for DL_ADC12_enableDMATrigger
    ti_msp_dl_config.o(.text.SYSCFG_DL_ADC_VOLTAGE_init) refers to ti_msp_dl_config.o(.text.DL_ADC12_enableConversions) for DL_ADC12_enableConversions
    ti_msp_dl_config.o(.text.SYSCFG_DL_ADC_VOLTAGE_init) refers to ti_msp_dl_config.o(.rodata.gADC_VOLTAGEClockConfig) for [Anonymous Symbol]
    ti_msp_dl_config.o(.ARM.exidx.text.SYSCFG_DL_ADC_VOLTAGE_init) refers to ti_msp_dl_config.o(.text.SYSCFG_DL_ADC_VOLTAGE_init) for [Anonymous Symbol]
    ti_msp_dl_config.o(.text.SYSCFG_DL_DMA_init) refers to ti_msp_dl_config.o(.text.SYSCFG_DL_DMA_CH0_init) for SYSCFG_DL_DMA_CH0_init
    ti_msp_dl_config.o(.ARM.exidx.text.SYSCFG_DL_DMA_init) refers to ti_msp_dl_config.o(.text.SYSCFG_DL_DMA_init) for [Anonymous Symbol]
    ti_msp_dl_config.o(.text.SYSCFG_DL_SYSTICK_init) refers to ti_msp_dl_config.o(.text.SysTick_Config) for SysTick_Config
    ti_msp_dl_config.o(.ARM.exidx.text.SYSCFG_DL_SYSTICK_init) refers to ti_msp_dl_config.o(.text.SYSCFG_DL_SYSTICK_init) for [Anonymous Symbol]
    ti_msp_dl_config.o(.ARM.exidx.text.DL_GPIO_reset) refers to ti_msp_dl_config.o(.text.DL_GPIO_reset) for [Anonymous Symbol]
    ti_msp_dl_config.o(.ARM.exidx.text.DL_Timer_reset) refers to ti_msp_dl_config.o(.text.DL_Timer_reset) for [Anonymous Symbol]
    ti_msp_dl_config.o(.ARM.exidx.text.DL_UART_reset) refers to ti_msp_dl_config.o(.text.DL_UART_reset) for [Anonymous Symbol]
    ti_msp_dl_config.o(.ARM.exidx.text.DL_ADC12_reset) refers to ti_msp_dl_config.o(.text.DL_ADC12_reset) for [Anonymous Symbol]
    ti_msp_dl_config.o(.ARM.exidx.text.DL_GPIO_enablePower) refers to ti_msp_dl_config.o(.text.DL_GPIO_enablePower) for [Anonymous Symbol]
    ti_msp_dl_config.o(.ARM.exidx.text.DL_Timer_enablePower) refers to ti_msp_dl_config.o(.text.DL_Timer_enablePower) for [Anonymous Symbol]
    ti_msp_dl_config.o(.ARM.exidx.text.DL_UART_enablePower) refers to ti_msp_dl_config.o(.text.DL_UART_enablePower) for [Anonymous Symbol]
    ti_msp_dl_config.o(.ARM.exidx.text.DL_ADC12_enablePower) refers to ti_msp_dl_config.o(.text.DL_ADC12_enablePower) for [Anonymous Symbol]
    ti_msp_dl_config.o(.ARM.exidx.text.DL_GPIO_initPeripheralOutputFunction) refers to ti_msp_dl_config.o(.text.DL_GPIO_initPeripheralOutputFunction) for [Anonymous Symbol]
    ti_msp_dl_config.o(.ARM.exidx.text.DL_GPIO_initPeripheralInputFunction) refers to ti_msp_dl_config.o(.text.DL_GPIO_initPeripheralInputFunction) for [Anonymous Symbol]
    ti_msp_dl_config.o(.ARM.exidx.text.DL_GPIO_initDigitalOutput) refers to ti_msp_dl_config.o(.text.DL_GPIO_initDigitalOutput) for [Anonymous Symbol]
    ti_msp_dl_config.o(.ARM.exidx.text.DL_GPIO_initDigitalInputFeatures) refers to ti_msp_dl_config.o(.text.DL_GPIO_initDigitalInputFeatures) for [Anonymous Symbol]
    ti_msp_dl_config.o(.ARM.exidx.text.DL_GPIO_clearPins) refers to ti_msp_dl_config.o(.text.DL_GPIO_clearPins) for [Anonymous Symbol]
    ti_msp_dl_config.o(.ARM.exidx.text.DL_GPIO_enableOutput) refers to ti_msp_dl_config.o(.text.DL_GPIO_enableOutput) for [Anonymous Symbol]
    ti_msp_dl_config.o(.ARM.exidx.text.DL_GPIO_setUpperPinsPolarity) refers to ti_msp_dl_config.o(.text.DL_GPIO_setUpperPinsPolarity) for [Anonymous Symbol]
    ti_msp_dl_config.o(.ARM.exidx.text.DL_GPIO_clearInterruptStatus) refers to ti_msp_dl_config.o(.text.DL_GPIO_clearInterruptStatus) for [Anonymous Symbol]
    ti_msp_dl_config.o(.ARM.exidx.text.DL_GPIO_enableInterrupt) refers to ti_msp_dl_config.o(.text.DL_GPIO_enableInterrupt) for [Anonymous Symbol]
    ti_msp_dl_config.o(.ARM.exidx.text.DL_SYSCTL_setBORThreshold) refers to ti_msp_dl_config.o(.text.DL_SYSCTL_setBORThreshold) for [Anonymous Symbol]
    ti_msp_dl_config.o(.text.DL_SYSCTL_setSYSOSCFreq) refers to ti_msp_dl_config.o(.text.DL_Common_updateReg) for DL_Common_updateReg
    ti_msp_dl_config.o(.ARM.exidx.text.DL_SYSCTL_setSYSOSCFreq) refers to ti_msp_dl_config.o(.text.DL_SYSCTL_setSYSOSCFreq) for [Anonymous Symbol]
    ti_msp_dl_config.o(.ARM.exidx.text.DL_SYSCTL_enableMFPCLK) refers to ti_msp_dl_config.o(.text.DL_SYSCTL_enableMFPCLK) for [Anonymous Symbol]
    ti_msp_dl_config.o(.ARM.exidx.text.__NVIC_SetPriority) refers to ti_msp_dl_config.o(.text.__NVIC_SetPriority) for [Anonymous Symbol]
    ti_msp_dl_config.o(.ARM.exidx.text.DL_Timer_enableInterrupt) refers to ti_msp_dl_config.o(.text.DL_Timer_enableInterrupt) for [Anonymous Symbol]
    ti_msp_dl_config.o(.ARM.exidx.text.DL_Timer_enableClock) refers to ti_msp_dl_config.o(.text.DL_Timer_enableClock) for [Anonymous Symbol]
    ti_msp_dl_config.o(.text.DL_UART_setOversampling) refers to ti_msp_dl_config.o(.text.DL_Common_updateReg) for DL_Common_updateReg
    ti_msp_dl_config.o(.ARM.exidx.text.DL_UART_setOversampling) refers to ti_msp_dl_config.o(.text.DL_UART_setOversampling) for [Anonymous Symbol]
    ti_msp_dl_config.o(.text.DL_UART_setBaudRateDivisor) refers to ti_msp_dl_config.o(.text.DL_Common_updateReg) for DL_Common_updateReg
    ti_msp_dl_config.o(.ARM.exidx.text.DL_UART_setBaudRateDivisor) refers to ti_msp_dl_config.o(.text.DL_UART_setBaudRateDivisor) for [Anonymous Symbol]
    ti_msp_dl_config.o(.ARM.exidx.text.DL_UART_enable) refers to ti_msp_dl_config.o(.text.DL_UART_enable) for [Anonymous Symbol]
    ti_msp_dl_config.o(.text.DL_ADC12_initSingleSample) refers to ti_msp_dl_config.o(.text.DL_Common_updateReg) for DL_Common_updateReg
    ti_msp_dl_config.o(.ARM.exidx.text.DL_ADC12_initSingleSample) refers to ti_msp_dl_config.o(.text.DL_ADC12_initSingleSample) for [Anonymous Symbol]
    ti_msp_dl_config.o(.ARM.exidx.text.DL_ADC12_configConversionMem) refers to ti_msp_dl_config.o(.text.DL_ADC12_configConversionMem) for [Anonymous Symbol]
    ti_msp_dl_config.o(.ARM.exidx.text.DL_ADC12_setSampleTime0) refers to ti_msp_dl_config.o(.text.DL_ADC12_setSampleTime0) for [Anonymous Symbol]
    ti_msp_dl_config.o(.ARM.exidx.text.DL_ADC12_enableDMA) refers to ti_msp_dl_config.o(.text.DL_ADC12_enableDMA) for [Anonymous Symbol]
    ti_msp_dl_config.o(.text.DL_ADC12_setDMASamplesCnt) refers to ti_msp_dl_config.o(.text.DL_Common_updateReg) for DL_Common_updateReg
    ti_msp_dl_config.o(.ARM.exidx.text.DL_ADC12_setDMASamplesCnt) refers to ti_msp_dl_config.o(.text.DL_ADC12_setDMASamplesCnt) for [Anonymous Symbol]
    ti_msp_dl_config.o(.ARM.exidx.text.DL_ADC12_enableDMATrigger) refers to ti_msp_dl_config.o(.text.DL_ADC12_enableDMATrigger) for [Anonymous Symbol]
    ti_msp_dl_config.o(.ARM.exidx.text.DL_ADC12_enableConversions) refers to ti_msp_dl_config.o(.text.DL_ADC12_enableConversions) for [Anonymous Symbol]
    ti_msp_dl_config.o(.text.SYSCFG_DL_DMA_CH0_init) refers to ti_msp_dl_config.o(.text.DL_DMA_setTransferSize) for DL_DMA_setTransferSize
    ti_msp_dl_config.o(.text.SYSCFG_DL_DMA_CH0_init) refers to dl_dma.o(.text.DL_DMA_initChannel) for DL_DMA_initChannel
    ti_msp_dl_config.o(.text.SYSCFG_DL_DMA_CH0_init) refers to ti_msp_dl_config.o(.rodata.gDMA_CH0Config) for [Anonymous Symbol]
    ti_msp_dl_config.o(.ARM.exidx.text.SYSCFG_DL_DMA_CH0_init) refers to ti_msp_dl_config.o(.text.SYSCFG_DL_DMA_CH0_init) for [Anonymous Symbol]
    ti_msp_dl_config.o(.ARM.exidx.text.DL_DMA_setTransferSize) refers to ti_msp_dl_config.o(.text.DL_DMA_setTransferSize) for [Anonymous Symbol]
    ti_msp_dl_config.o(.text.SysTick_Config) refers to ti_msp_dl_config.o(.text.__NVIC_SetPriority) for __NVIC_SetPriority
    ti_msp_dl_config.o(.ARM.exidx.text.SysTick_Config) refers to ti_msp_dl_config.o(.text.SysTick_Config) for [Anonymous Symbol]
    ti_msp_dl_config.o(.ARM.exidx.text.DL_Common_updateReg) refers to ti_msp_dl_config.o(.text.DL_Common_updateReg) for [Anonymous Symbol]
    adc.o(.text.adc_getValue) refers to memseta.o(.text) for __aeabi_memclr
    adc.o(.text.adc_getValue) refers to uidiv_div0.o(.text) for __aeabi_uidiv
    adc.o(.text.adc_getValue) refers to adc.o(.bss.ADC_VALUE) for ADC_VALUE
    adc.o(.ARM.exidx.text.adc_getValue) refers to adc.o(.text.adc_getValue) for [Anonymous Symbol]
    delay.o(.text.SysTick_Handler) refers to delay.o(.text.Tick_SysTickCallback) for Tick_SysTickCallback
    delay.o(.ARM.exidx.text.SysTick_Handler) refers to delay.o(.text.SysTick_Handler) for [Anonymous Symbol]
    delay.o(.text.Tick_SysTickCallback) refers to delay.o(.bss.Tick) for Tick
    delay.o(.ARM.exidx.text.Tick_SysTickCallback) refers to delay.o(.text.Tick_SysTickCallback) for [Anonymous Symbol]
    delay.o(.ARM.exidx.text.delay_us) refers to delay.o(.text.delay_us) for [Anonymous Symbol]
    delay.o(.text.Tick_delay) refers to delay.o(.bss.Tick) for Tick
    delay.o(.ARM.exidx.text.Tick_delay) refers to delay.o(.text.Tick_delay) for [Anonymous Symbol]
    no_mcu_ganv_grayscale_sensor.o(.text.Get_Analog_value) refers to no_mcu_ganv_grayscale_sensor.o(.text.DL_GPIO_setPins) for DL_GPIO_setPins
    no_mcu_ganv_grayscale_sensor.o(.text.Get_Analog_value) refers to no_mcu_ganv_grayscale_sensor.o(.text.DL_GPIO_clearPins) for DL_GPIO_clearPins
    no_mcu_ganv_grayscale_sensor.o(.text.Get_Analog_value) refers to delay.o(.text.delay_us) for delay_us
    no_mcu_ganv_grayscale_sensor.o(.text.Get_Analog_value) refers to adc.o(.text.adc_getValue) for adc_getValue
    no_mcu_ganv_grayscale_sensor.o(.ARM.exidx.text.Get_Analog_value) refers to no_mcu_ganv_grayscale_sensor.o(.text.Get_Analog_value) for [Anonymous Symbol]
    no_mcu_ganv_grayscale_sensor.o(.ARM.exidx.text.DL_GPIO_setPins) refers to no_mcu_ganv_grayscale_sensor.o(.text.DL_GPIO_setPins) for [Anonymous Symbol]
    no_mcu_ganv_grayscale_sensor.o(.ARM.exidx.text.DL_GPIO_clearPins) refers to no_mcu_ganv_grayscale_sensor.o(.text.DL_GPIO_clearPins) for [Anonymous Symbol]
    no_mcu_ganv_grayscale_sensor.o(.ARM.exidx.text.convertAnalogToDigital) refers to no_mcu_ganv_grayscale_sensor.o(.text.convertAnalogToDigital) for [Anonymous Symbol]
    no_mcu_ganv_grayscale_sensor.o(.text.normalizeAnalogValues) refers to dflti.o(.text) for __aeabi_i2d
    no_mcu_ganv_grayscale_sensor.o(.text.normalizeAnalogValues) refers to dmul.o(.text) for __aeabi_dmul
    no_mcu_ganv_grayscale_sensor.o(.text.normalizeAnalogValues) refers to dfixi.o(.text) for __aeabi_d2iz
    no_mcu_ganv_grayscale_sensor.o(.text.normalizeAnalogValues) refers to dcmple.o(.text) for __aeabi_dcmple
    no_mcu_ganv_grayscale_sensor.o(.ARM.exidx.text.normalizeAnalogValues) refers to no_mcu_ganv_grayscale_sensor.o(.text.normalizeAnalogValues) for [Anonymous Symbol]
    no_mcu_ganv_grayscale_sensor.o(.ARM.exidx.text.No_MCU_Ganv_Sensor_Init_Frist) refers to no_mcu_ganv_grayscale_sensor.o(.text.No_MCU_Ganv_Sensor_Init_Frist) for [Anonymous Symbol]
    no_mcu_ganv_grayscale_sensor.o(.text.No_MCU_Ganv_Sensor_Init) refers to no_mcu_ganv_grayscale_sensor.o(.text.No_MCU_Ganv_Sensor_Init_Frist) for No_MCU_Ganv_Sensor_Init_Frist
    no_mcu_ganv_grayscale_sensor.o(.text.No_MCU_Ganv_Sensor_Init) refers to uidiv_div0.o(.text) for __aeabi_uidiv
    no_mcu_ganv_grayscale_sensor.o(.text.No_MCU_Ganv_Sensor_Init) refers to dfltui.o(.text) for __aeabi_ui2d
    no_mcu_ganv_grayscale_sensor.o(.text.No_MCU_Ganv_Sensor_Init) refers to dadd.o(.text) for __aeabi_dsub
    no_mcu_ganv_grayscale_sensor.o(.text.No_MCU_Ganv_Sensor_Init) refers to ddiv.o(.text) for __aeabi_ddiv
    no_mcu_ganv_grayscale_sensor.o(.ARM.exidx.text.No_MCU_Ganv_Sensor_Init) refers to no_mcu_ganv_grayscale_sensor.o(.text.No_MCU_Ganv_Sensor_Init) for [Anonymous Symbol]
    no_mcu_ganv_grayscale_sensor.o(.text.No_Mcu_Ganv_Sensor_Task_Without_tick) refers to no_mcu_ganv_grayscale_sensor.o(.text.Get_Analog_value) for Get_Analog_value
    no_mcu_ganv_grayscale_sensor.o(.text.No_Mcu_Ganv_Sensor_Task_Without_tick) refers to no_mcu_ganv_grayscale_sensor.o(.text.convertAnalogToDigital) for convertAnalogToDigital
    no_mcu_ganv_grayscale_sensor.o(.text.No_Mcu_Ganv_Sensor_Task_Without_tick) refers to no_mcu_ganv_grayscale_sensor.o(.text.normalizeAnalogValues) for normalizeAnalogValues
    no_mcu_ganv_grayscale_sensor.o(.ARM.exidx.text.No_Mcu_Ganv_Sensor_Task_Without_tick) refers to no_mcu_ganv_grayscale_sensor.o(.text.No_Mcu_Ganv_Sensor_Task_Without_tick) for [Anonymous Symbol]
    no_mcu_ganv_grayscale_sensor.o(.text.No_Mcu_Ganv_Sensor_Task_With_tick) refers to no_mcu_ganv_grayscale_sensor.o(.text.Get_Analog_value) for Get_Analog_value
    no_mcu_ganv_grayscale_sensor.o(.text.No_Mcu_Ganv_Sensor_Task_With_tick) refers to no_mcu_ganv_grayscale_sensor.o(.text.convertAnalogToDigital) for convertAnalogToDigital
    no_mcu_ganv_grayscale_sensor.o(.text.No_Mcu_Ganv_Sensor_Task_With_tick) refers to no_mcu_ganv_grayscale_sensor.o(.text.normalizeAnalogValues) for normalizeAnalogValues
    no_mcu_ganv_grayscale_sensor.o(.ARM.exidx.text.No_Mcu_Ganv_Sensor_Task_With_tick) refers to no_mcu_ganv_grayscale_sensor.o(.text.No_Mcu_Ganv_Sensor_Task_With_tick) for [Anonymous Symbol]
    no_mcu_ganv_grayscale_sensor.o(.ARM.exidx.text.Task_tick) refers to no_mcu_ganv_grayscale_sensor.o(.text.Task_tick) for [Anonymous Symbol]
    no_mcu_ganv_grayscale_sensor.o(.ARM.exidx.text.Get_Digtal_For_User) refers to no_mcu_ganv_grayscale_sensor.o(.text.Get_Digtal_For_User) for [Anonymous Symbol]
    no_mcu_ganv_grayscale_sensor.o(.text.Get_Normalize_For_User) refers to memcpya.o(.text) for __aeabi_memcpy
    no_mcu_ganv_grayscale_sensor.o(.ARM.exidx.text.Get_Normalize_For_User) refers to no_mcu_ganv_grayscale_sensor.o(.text.Get_Normalize_For_User) for [Anonymous Symbol]
    no_mcu_ganv_grayscale_sensor.o(.text.Get_Anolog_Value) refers to memcpya.o(.text) for __aeabi_memcpy
    no_mcu_ganv_grayscale_sensor.o(.ARM.exidx.text.Get_Anolog_Value) refers to no_mcu_ganv_grayscale_sensor.o(.text.Get_Anolog_Value) for [Anonymous Symbol]
    key.o(.text.GROUP1_IRQHandler) refers to key.o(.text.DL_GPIO_getPendingInterrupt) for DL_GPIO_getPendingInterrupt
    key.o(.text.GROUP1_IRQHandler) refers to key.o(.text.DL_GPIO_readPins) for DL_GPIO_readPins
    key.o(.text.GROUP1_IRQHandler) refers to delay.o(.bss.Tick) for Tick
    key.o(.text.GROUP1_IRQHandler) refers to key.o(.bss.last_key_time) for last_key_time
    key.o(.text.GROUP1_IRQHandler) refers to key.o(.bss.key_pressed) for key_pressed
    key.o(.text.GROUP1_IRQHandler) refers to key.o(.bss.key_start_pressed) for key_start_pressed
    key.o(.ARM.exidx.text.GROUP1_IRQHandler) refers to key.o(.text.GROUP1_IRQHandler) for [Anonymous Symbol]
    key.o(.ARM.exidx.text.DL_GPIO_getPendingInterrupt) refers to key.o(.text.DL_GPIO_getPendingInterrupt) for [Anonymous Symbol]
    key.o(.ARM.exidx.text.DL_GPIO_readPins) refers to key.o(.text.DL_GPIO_readPins) for [Anonymous Symbol]
    pid.o(.text.Pid_Yaw) refers to fflti.o(.text) for __aeabi_i2f
    pid.o(.text.Pid_Yaw) refers to fadd.o(.text) for __aeabi_fsub
    pid.o(.text.Pid_Yaw) refers to ffixi.o(.text) for __aeabi_f2iz
    pid.o(.text.Pid_Yaw) refers to pid.o(.bss.result_angle) for result_angle
    pid.o(.text.Pid_Yaw) refers to pid.o(.bss.Yaw_Now_Correct) for Yaw_Now_Correct
    pid.o(.text.Pid_Yaw) refers to pid.o(.bss.Err_Yaw) for Err_Yaw
    pid.o(.text.Pid_Yaw) refers to pid.o(.bss.Integral_Yaw) for Integral_Yaw
    pid.o(.text.Pid_Yaw) refers to pid.o(.data.Kp_Yaw) for Kp_Yaw
    pid.o(.text.Pid_Yaw) refers to pid.o(.data.Kd_Yaw) for Kd_Yaw
    pid.o(.text.Pid_Yaw) refers to pid.o(.bss.LastErr_Yaw) for LastErr_Yaw
    pid.o(.text.Pid_Yaw) refers to pid.o(.bss.Ki_Yaw) for Ki_Yaw
    pid.o(.text.Pid_Yaw) refers to pid.o(.bss.Output_Yaw) for Output_Yaw
    pid.o(.text.Pid_Yaw) refers to pid.o(.data.max) for max
    pid.o(.ARM.exidx.text.Pid_Yaw) refers to pid.o(.text.Pid_Yaw) for [Anonymous Symbol]
    l298n.o(.text.Motor_SetDuty_A) refers to l298n.o(.data.motorDuty_A) for motorDuty_A
    l298n.o(.ARM.exidx.text.Motor_SetDuty_A) refers to l298n.o(.text.Motor_SetDuty_A) for [Anonymous Symbol]
    l298n.o(.text.Motor_SetDuty_B) refers to l298n.o(.data.motorDuty_B) for motorDuty_B
    l298n.o(.ARM.exidx.text.Motor_SetDuty_B) refers to l298n.o(.text.Motor_SetDuty_B) for [Anonymous Symbol]
    l298n.o(.text.Motor_UpdatePWM_A) refers to uidiv_div0.o(.text) for __aeabi_uidivmod
    l298n.o(.text.Motor_UpdatePWM_A) refers to l298n.o(.text.DL_GPIO_clearPins) for DL_GPIO_clearPins
    l298n.o(.text.Motor_UpdatePWM_A) refers to l298n.o(.text.DL_GPIO_setPins) for DL_GPIO_setPins
    l298n.o(.text.Motor_UpdatePWM_A) refers to l298n.o(.bss.pwmCounter_A) for pwmCounter_A
    l298n.o(.text.Motor_UpdatePWM_A) refers to l298n.o(.data.motorDuty_A) for motorDuty_A
    l298n.o(.ARM.exidx.text.Motor_UpdatePWM_A) refers to l298n.o(.text.Motor_UpdatePWM_A) for [Anonymous Symbol]
    l298n.o(.ARM.exidx.text.DL_GPIO_clearPins) refers to l298n.o(.text.DL_GPIO_clearPins) for [Anonymous Symbol]
    l298n.o(.ARM.exidx.text.DL_GPIO_setPins) refers to l298n.o(.text.DL_GPIO_setPins) for [Anonymous Symbol]
    l298n.o(.text.TIMG0_IRQHandler) refers to l298n.o(.text.Motor_UpdatePWM_A) for Motor_UpdatePWM_A
    l298n.o(.text.TIMG0_IRQHandler) refers to l298n.o(.text.Motor_UpdatePWM_B) for Motor_UpdatePWM_B
    l298n.o(.ARM.exidx.text.TIMG0_IRQHandler) refers to l298n.o(.text.TIMG0_IRQHandler) for [Anonymous Symbol]
    l298n.o(.text.Motor_UpdatePWM_B) refers to uidiv_div0.o(.text) for __aeabi_uidivmod
    l298n.o(.text.Motor_UpdatePWM_B) refers to l298n.o(.text.DL_GPIO_setPins) for DL_GPIO_setPins
    l298n.o(.text.Motor_UpdatePWM_B) refers to l298n.o(.text.DL_GPIO_clearPins) for DL_GPIO_clearPins
    l298n.o(.text.Motor_UpdatePWM_B) refers to l298n.o(.bss.pwmCounter_B) for pwmCounter_B
    l298n.o(.text.Motor_UpdatePWM_B) refers to l298n.o(.data.motorDuty_B) for motorDuty_B
    l298n.o(.ARM.exidx.text.Motor_UpdatePWM_B) refers to l298n.o(.text.Motor_UpdatePWM_B) for [Anonymous Symbol]
    l298n.o(.text.Motor_Control) refers to pid.o(.text.Pid_Yaw) for Pid_Yaw
    l298n.o(.text.Motor_Control) refers to l298n.o(.text.Motor_SetDuty_B) for Motor_SetDuty_B
    l298n.o(.text.Motor_Control) refers to l298n.o(.text.Motor_SetDuty_A) for Motor_SetDuty_A
    l298n.o(.text.Motor_Control) refers to l298n.o(.bss.Tarangle) for Tarangle
    l298n.o(.text.Motor_Control) refers to l298n.o(.data.K_V) for K_V
    l298n.o(.text.Motor_Control) refers to pid.o(.bss.result_angle) for result_angle
    l298n.o(.text.Motor_Control) refers to l298n.o(.bss.Speed_Set) for Speed_Set
    l298n.o(.text.Motor_Control) refers to main.o(.bss.Digtal) for Digtal
    l298n.o(.text.Motor_Control) refers to pid.o(.bss.Output_Yaw) for Output_Yaw
    l298n.o(.text.Motor_Control) refers to l298n.o(.bss.pwmL) for pwmL
    l298n.o(.text.Motor_Control) refers to l298n.o(.bss.pwmR) for pwmR
    l298n.o(.text.Motor_Control) refers to l298n.o(.bss.SpeedR) for SpeedR
    l298n.o(.text.Motor_Control) refers to l298n.o(.bss.SpeedL) for SpeedL
    l298n.o(.ARM.exidx.text.Motor_Control) refers to l298n.o(.text.Motor_Control) for [Anonymous Symbol]
    retarget_io.o(.text.fputc) refers to retarget_io.o(.text.stdout_putchar) for stdout_putchar
    retarget_io.o(.text.fputc) refers to retarget_io.o(.text.stderr_putchar) for stderr_putchar
    retarget_io.o(.text.fputc) refers to stdout.o(.data) for __stdout
    retarget_io.o(.text.fputc) refers to stderr.o(.data) for __stderr
    retarget_io.o(.ARM.exidx.text.fputc) refers to retarget_io.o(.text.fputc) for [Anonymous Symbol]
    retarget_io.o(.ARM.exidx.text.stdout_putchar) refers to retarget_io.o(.text.stdout_putchar) for [Anonymous Symbol]
    retarget_io.o(.ARM.exidx.text.stderr_putchar) refers to retarget_io.o(.text.stderr_putchar) for [Anonymous Symbol]
    retarget_io.o(.text.fgetc) refers to retarget_io.o(.text.stdin_getchar) for stdin_getchar
    retarget_io.o(.text.fgetc) refers to stdin.o(.data) for __stdin
    retarget_io.o(.text.fgetc) refers to retarget_io.o(.bss.getchar_undo) for [Anonymous Symbol]
    retarget_io.o(.text.fgetc) refers to retarget_io.o(.data.getchar_ch) for [Anonymous Symbol]
    retarget_io.o(.ARM.exidx.text.fgetc) refers to retarget_io.o(.text.fgetc) for [Anonymous Symbol]
    retarget_io.o(.ARM.exidx.text.stdin_getchar) refers to retarget_io.o(.text.stdin_getchar) for [Anonymous Symbol]
    retarget_io.o(.text.__backspace) refers to stdin.o(.data) for __stdin
    retarget_io.o(.text.__backspace) refers to retarget_io.o(.data.getchar_ch) for [Anonymous Symbol]
    retarget_io.o(.text.__backspace) refers to retarget_io.o(.bss.getchar_undo) for [Anonymous Symbol]
    retarget_io.o(.ARM.exidx.text.__backspace) refers to retarget_io.o(.text.__backspace) for [Anonymous Symbol]
    retarget_io.o(.text.__aeabi_assert) refers to fputs.o(i.fputs) for fputs
    retarget_io.o(.text.__aeabi_assert) refers to idiv_div0.o(.text) for __aeabi_idivmod
    retarget_io.o(.text.__aeabi_assert) refers to retarget_io.o(.text.abort) for abort
    retarget_io.o(.text.__aeabi_assert) refers to retarget_io.o(.rodata.str1.1) for [Anonymous Symbol]
    retarget_io.o(.text.__aeabi_assert) refers to stderr.o(.data) for __stderr
    retarget_io.o(.ARM.exidx.text.__aeabi_assert) refers to retarget_io.o(.text.__aeabi_assert) for [Anonymous Symbol]
    retarget_io.o(.ARM.exidx.text.abort) refers to retarget_io.o(.text.abort) for [Anonymous Symbol]
    dl_adc12.o(.ARM.exidx.text.DL_ADC12_setClockConfig) refers to dl_adc12.o(.text.DL_ADC12_setClockConfig) for [Anonymous Symbol]
    dl_adc12.o(.ARM.exidx.text.DL_ADC12_getClockConfig) refers to dl_adc12.o(.text.DL_ADC12_getClockConfig) for [Anonymous Symbol]
    dl_common.o(.ARM.exidx.text.DL_Common_delayCycles) refers to dl_common.o(.text.DL_Common_delayCycles) for [Anonymous Symbol]
    dl_dma.o(.ARM.exidx.text.DL_DMA_initChannel) refers to dl_dma.o(.text.DL_DMA_initChannel) for [Anonymous Symbol]
    dl_timer.o(.ARM.exidx.text.DL_Timer_setClockConfig) refers to dl_timer.o(.text.DL_Timer_setClockConfig) for [Anonymous Symbol]
    dl_timer.o(.ARM.exidx.text.DL_Timer_getClockConfig) refers to dl_timer.o(.text.DL_Timer_getClockConfig) for [Anonymous Symbol]
    dl_timer.o(.ARM.exidx.text.DL_Timer_initTimerMode) refers to dl_timer.o(.text.DL_Timer_initTimerMode) for [Anonymous Symbol]
    dl_timer.o(.ARM.exidx.text.DL_Timer_setCaptureCompareValue) refers to dl_timer.o(.text.DL_Timer_setCaptureCompareValue) for [Anonymous Symbol]
    dl_timer.o(.ARM.exidx.text.DL_Timer_setCaptureCompareCtl) refers to dl_timer.o(.text.DL_Timer_setCaptureCompareCtl) for [Anonymous Symbol]
    dl_timer.o(.text.DL_Timer_initCaptureMode) refers to dl_timer.o(.rodata..Lswitch.table.DL_Timer_initCompareMode) for [Anonymous Symbol]
    dl_timer.o(.ARM.exidx.text.DL_Timer_initCaptureMode) refers to dl_timer.o(.text.DL_Timer_initCaptureMode) for [Anonymous Symbol]
    dl_timer.o(.ARM.exidx.text.DL_Timer_setCaptureCompareInput) refers to dl_timer.o(.text.DL_Timer_setCaptureCompareInput) for [Anonymous Symbol]
    dl_timer.o(.ARM.exidx.text.DL_Timer_initCaptureTriggerMode) refers to dl_timer.o(.text.DL_Timer_initCaptureTriggerMode) for [Anonymous Symbol]
    dl_timer.o(.text.DL_Timer_initCaptureCombinedMode) refers to dl_timer.o(.rodata..Lswitch.table.DL_Timer_initCompareMode) for [Anonymous Symbol]
    dl_timer.o(.ARM.exidx.text.DL_Timer_initCaptureCombinedMode) refers to dl_timer.o(.text.DL_Timer_initCaptureCombinedMode) for [Anonymous Symbol]
    dl_timer.o(.text.DL_Timer_initCompareMode) refers to dl_timer.o(.rodata..Lswitch.table.DL_Timer_initCompareMode) for [Anonymous Symbol]
    dl_timer.o(.ARM.exidx.text.DL_Timer_initCompareMode) refers to dl_timer.o(.text.DL_Timer_initCompareMode) for [Anonymous Symbol]
    dl_timer.o(.ARM.exidx.text.DL_Timer_initCompareTriggerMode) refers to dl_timer.o(.text.DL_Timer_initCompareTriggerMode) for [Anonymous Symbol]
    dl_timer.o(.ARM.exidx.text.DL_Timer_initPWMMode) refers to dl_timer.o(.text.DL_Timer_initPWMMode) for [Anonymous Symbol]
    dl_timer.o(.ARM.exidx.text.DL_Timer_setCaptureCompareAction) refers to dl_timer.o(.text.DL_Timer_setCaptureCompareAction) for [Anonymous Symbol]
    dl_timer.o(.ARM.exidx.text.DL_Timer_setCaptureCompareOutCtl) refers to dl_timer.o(.text.DL_Timer_setCaptureCompareOutCtl) for [Anonymous Symbol]
    dl_timer.o(.ARM.exidx.text.DL_Timer_getCaptureCompareValue) refers to dl_timer.o(.text.DL_Timer_getCaptureCompareValue) for [Anonymous Symbol]
    dl_timer.o(.ARM.exidx.text.DL_Timer_getCaptureCompareCtl) refers to dl_timer.o(.text.DL_Timer_getCaptureCompareCtl) for [Anonymous Symbol]
    dl_timer.o(.ARM.exidx.text.DL_Timer_enableSuppressionOfCompEvent) refers to dl_timer.o(.text.DL_Timer_enableSuppressionOfCompEvent) for [Anonymous Symbol]
    dl_timer.o(.ARM.exidx.text.DL_Timer_disableSuppressionOfCompEvent) refers to dl_timer.o(.text.DL_Timer_disableSuppressionOfCompEvent) for [Anonymous Symbol]
    dl_timer.o(.ARM.exidx.text.DL_Timer_setCaptCompUpdateMethod) refers to dl_timer.o(.text.DL_Timer_setCaptCompUpdateMethod) for [Anonymous Symbol]
    dl_timer.o(.ARM.exidx.text.DL_Timer_getCaptCompUpdateMethod) refers to dl_timer.o(.text.DL_Timer_getCaptCompUpdateMethod) for [Anonymous Symbol]
    dl_timer.o(.ARM.exidx.text.DL_Timer_getCaptureCompareOutCtl) refers to dl_timer.o(.text.DL_Timer_getCaptureCompareOutCtl) for [Anonymous Symbol]
    dl_timer.o(.ARM.exidx.text.DL_Timer_getCaptureCompareAction) refers to dl_timer.o(.text.DL_Timer_getCaptureCompareAction) for [Anonymous Symbol]
    dl_timer.o(.ARM.exidx.text.DL_Timer_overrideCCPOut) refers to dl_timer.o(.text.DL_Timer_overrideCCPOut) for [Anonymous Symbol]
    dl_timer.o(.ARM.exidx.text.DL_Timer_getCaptureCompareInput) refers to dl_timer.o(.text.DL_Timer_getCaptureCompareInput) for [Anonymous Symbol]
    dl_timer.o(.ARM.exidx.text.DL_Timer_setCaptureCompareInputFilter) refers to dl_timer.o(.text.DL_Timer_setCaptureCompareInputFilter) for [Anonymous Symbol]
    dl_timer.o(.ARM.exidx.text.DL_Timer_getCaptureCompareInputFilter) refers to dl_timer.o(.text.DL_Timer_getCaptureCompareInputFilter) for [Anonymous Symbol]
    dl_timer.o(.ARM.exidx.text.DL_Timer_enableCaptureCompareInputFilter) refers to dl_timer.o(.text.DL_Timer_enableCaptureCompareInputFilter) for [Anonymous Symbol]
    dl_timer.o(.ARM.exidx.text.DL_Timer_disableCaptureCompareInputFilter) refers to dl_timer.o(.text.DL_Timer_disableCaptureCompareInputFilter) for [Anonymous Symbol]
    dl_timer.o(.ARM.exidx.text.DL_Timer_isCaptureCompareInputFilterEnabled) refers to dl_timer.o(.text.DL_Timer_isCaptureCompareInputFilterEnabled) for [Anonymous Symbol]
    dl_timer.o(.ARM.exidx.text.DL_Timer_saveConfiguration) refers to dl_timer.o(.text.DL_Timer_saveConfiguration) for [Anonymous Symbol]
    dl_timer.o(.ARM.exidx.text.DL_Timer_restoreConfiguration) refers to dl_timer.o(.text.DL_Timer_restoreConfiguration) for [Anonymous Symbol]
    dl_timer.o(.ARM.exidx.text.DL_Timer_configQEIHallInputMode) refers to dl_timer.o(.text.DL_Timer_configQEIHallInputMode) for [Anonymous Symbol]
    dl_uart.o(.ARM.exidx.text.DL_UART_init) refers to dl_uart.o(.text.DL_UART_init) for [Anonymous Symbol]
    dl_uart.o(.ARM.exidx.text.DL_UART_setClockConfig) refers to dl_uart.o(.text.DL_UART_setClockConfig) for [Anonymous Symbol]
    dl_uart.o(.ARM.exidx.text.DL_UART_getClockConfig) refers to dl_uart.o(.text.DL_UART_getClockConfig) for [Anonymous Symbol]
    dl_uart.o(.text.DL_UART_configBaudRate) refers to uidiv_div0.o(.text) for __aeabi_uidiv
    dl_uart.o(.ARM.exidx.text.DL_UART_configBaudRate) refers to dl_uart.o(.text.DL_UART_configBaudRate) for [Anonymous Symbol]
    dl_uart.o(.ARM.exidx.text.DL_UART_configIrDAMode) refers to dl_uart.o(.text.DL_UART_configIrDAMode) for [Anonymous Symbol]
    dl_uart.o(.ARM.exidx.text.DL_UART_setIrDAPulseLength) refers to dl_uart.o(.text.DL_UART_setIrDAPulseLength) for [Anonymous Symbol]
    dl_uart.o(.ARM.exidx.text.DL_UART_receiveDataBlocking) refers to dl_uart.o(.text.DL_UART_receiveDataBlocking) for [Anonymous Symbol]
    dl_uart.o(.ARM.exidx.text.DL_UART_transmitDataBlocking) refers to dl_uart.o(.text.DL_UART_transmitDataBlocking) for [Anonymous Symbol]
    dl_uart.o(.ARM.exidx.text.DL_UART_receiveDataCheck) refers to dl_uart.o(.text.DL_UART_receiveDataCheck) for [Anonymous Symbol]
    dl_uart.o(.ARM.exidx.text.DL_UART_transmitDataCheck) refers to dl_uart.o(.text.DL_UART_transmitDataCheck) for [Anonymous Symbol]
    dl_uart.o(.ARM.exidx.text.DL_UART_drainRXFIFO) refers to dl_uart.o(.text.DL_UART_drainRXFIFO) for [Anonymous Symbol]
    dl_uart.o(.ARM.exidx.text.DL_UART_fillTXFIFO) refers to dl_uart.o(.text.DL_UART_fillTXFIFO) for [Anonymous Symbol]
    dl_uart.o(.ARM.exidx.text.DL_UART_Main_saveConfiguration) refers to dl_uart.o(.text.DL_UART_Main_saveConfiguration) for [Anonymous Symbol]
    dl_uart.o(.ARM.exidx.text.DL_UART_Main_restoreConfiguration) refers to dl_uart.o(.text.DL_UART_Main_restoreConfiguration) for [Anonymous Symbol]
    dl_uart.o(.ARM.exidx.text.DL_UART_Extend_saveConfiguration) refers to dl_uart.o(.text.DL_UART_Extend_saveConfiguration) for [Anonymous Symbol]
    dl_uart.o(.ARM.exidx.text.DL_UART_Extend_restoreConfiguration) refers to dl_uart.o(.text.DL_UART_Extend_restoreConfiguration) for [Anonymous Symbol]
    entry.o(.ARM.Collect$$$$00000000) refers (Special) to entry10a.o(.ARM.Collect$$$$0000000D) for __rt_final_cpp
    entry.o(.ARM.Collect$$$$00000000) refers (Special) to entry11a.o(.ARM.Collect$$$$0000000F) for __rt_final_exit
    entry.o(.ARM.Collect$$$$00000000) refers (Special) to entry7b.o(.ARM.Collect$$$$00000008) for _main_clock
    entry.o(.ARM.Collect$$$$00000000) refers (Special) to entry8b.o(.ARM.Collect$$$$0000000A) for _main_cpp_init
    entry.o(.ARM.Collect$$$$00000000) refers (Special) to entry9a.o(.ARM.Collect$$$$0000000B) for _main_init
    entry.o(.ARM.Collect$$$$00000000) refers (Special) to entry5.o(.ARM.Collect$$$$00000004) for _main_scatterload
    entry.o(.ARM.Collect$$$$00000000) refers (Special) to entry2.o(.ARM.Collect$$$$00000001) for _main_stk
    fputs.o(i.fputs) refers to main.o(.text.fputc) for fputc
    fputs_e.o(.text) refers to main.o(.text.fputc) for fputc
    idiv.o(.text) refers to uidiv_div0.o(.text) for __aeabi_uidivmod
    printfa.o(i.__0fprintf) refers (Special) to iusefp.o(.text) for __I$use$fp
    printfa.o(i.__0fprintf) refers to printfa.o(i._printf_core) for _printf_core
    printfa.o(i.__0fprintf) refers to main.o(.text.fputc) for fputc
    printfa.o(i.__0printf) refers (Special) to iusefp.o(.text) for __I$use$fp
    printfa.o(i.__0printf) refers to printfa.o(i._printf_core) for _printf_core
    printfa.o(i.__0printf) refers to main.o(.text.fputc) for fputc
    printfa.o(i.__0printf) refers to stdout.o(.data) for __stdout
    printfa.o(i.__0snprintf) refers (Special) to iusefp.o(.text) for __I$use$fp
    printfa.o(i.__0snprintf) refers to printfa.o(i._printf_core) for _printf_core
    printfa.o(i.__0snprintf) refers to printfa.o(i._snputc) for _snputc
    printfa.o(i.__0sprintf) refers (Special) to iusefp.o(.text) for __I$use$fp
    printfa.o(i.__0sprintf) refers to printfa.o(i._printf_core) for _printf_core
    printfa.o(i.__0sprintf) refers to printfa.o(i._sputc) for _sputc
    printfa.o(i.__0vfprintf) refers (Special) to iusefp.o(.text) for __I$use$fp
    printfa.o(i.__0vfprintf) refers to printfa.o(i._printf_core) for _printf_core
    printfa.o(i.__0vfprintf) refers to main.o(.text.fputc) for fputc
    printfa.o(i.__0vprintf) refers (Special) to iusefp.o(.text) for __I$use$fp
    printfa.o(i.__0vprintf) refers to printfa.o(i._printf_core) for _printf_core
    printfa.o(i.__0vprintf) refers to main.o(.text.fputc) for fputc
    printfa.o(i.__0vprintf) refers to stdout.o(.data) for __stdout
    printfa.o(i.__0vsnprintf) refers (Special) to iusefp.o(.text) for __I$use$fp
    printfa.o(i.__0vsnprintf) refers to printfa.o(i._printf_core) for _printf_core
    printfa.o(i.__0vsnprintf) refers to printfa.o(i._snputc) for _snputc
    printfa.o(i.__0vsprintf) refers (Special) to iusefp.o(.text) for __I$use$fp
    printfa.o(i.__0vsprintf) refers to printfa.o(i._printf_core) for _printf_core
    printfa.o(i.__0vsprintf) refers to printfa.o(i._sputc) for _sputc
    printfa.o(i._fp_digits) refers (Special) to iusefp.o(.text) for __I$use$fp
    printfa.o(i._fp_digits) refers to dmul.o(.text) for __aeabi_dmul
    printfa.o(i._fp_digits) refers to ddiv.o(.text) for __aeabi_ddiv
    printfa.o(i._fp_digits) refers to cdrcmple.o(.text) for __aeabi_cdrcmple
    printfa.o(i._fp_digits) refers to dadd.o(.text) for __aeabi_dadd
    printfa.o(i._fp_digits) refers to dfixul.o(.text) for __aeabi_d2ulz
    printfa.o(i._fp_digits) refers to uldiv.o(.text) for __aeabi_uldivmod
    printfa.o(i._printf_core) refers (Special) to iusefp.o(.text) for __I$use$fp
    printfa.o(i._printf_core) refers to printfa.o(i._printf_pre_padding) for _printf_pre_padding
    printfa.o(i._printf_core) refers to uldiv.o(.text) for __aeabi_uldivmod
    printfa.o(i._printf_core) refers to printfa.o(i._printf_post_padding) for _printf_post_padding
    printfa.o(i._printf_core) refers to printfa.o(i._fp_digits) for _fp_digits
    printfa.o(i._printf_core) refers to uidiv_div0.o(.text) for __aeabi_uidivmod
    printfa.o(i._printf_post_padding) refers (Special) to iusefp.o(.text) for __I$use$fp
    printfa.o(i._printf_pre_padding) refers (Special) to iusefp.o(.text) for __I$use$fp
    printfa.o(i._snputc) refers (Special) to iusefp.o(.text) for __I$use$fp
    printfa.o(i._sputc) refers (Special) to iusefp.o(.text) for __I$use$fp
    fadd.o(.text) refers (Special) to iusefp.o(.text) for __I$use$fp
    fadd.o(.text) refers to fepilogue.o(.text) for _float_epilogue
    dadd.o(.text) refers (Special) to iusefp.o(.text) for __I$use$fp
    dadd.o(.text) refers to llshl.o(.text) for __aeabi_llsl
    dadd.o(.text) refers to llsshr.o(.text) for __aeabi_lasr
    dadd.o(.text) refers to depilogue.o(.text) for _double_epilogue
    dmul.o(.text) refers (Special) to iusefp.o(.text) for __I$use$fp
    dmul.o(.text) refers to depilogue.o(.text) for _double_epilogue
    ddiv.o(.text) refers (Special) to iusefp.o(.text) for __I$use$fp
    ddiv.o(.text) refers to depilogue.o(.text) for _double_round
    dcmple.o(.text) refers (Special) to iusefp.o(.text) for __I$use$fp
    fflti.o(.text) refers (Special) to iusefp.o(.text) for __I$use$fp
    fflti.o(.text) refers to fepilogue.o(.text) for _float_epilogue
    dflti.o(.text) refers (Special) to iusefp.o(.text) for __I$use$fp
    dflti.o(.text) refers to depilogue.o(.text) for _double_epilogue
    dfltui.o(.text) refers (Special) to iusefp.o(.text) for __I$use$fp
    dfltui.o(.text) refers to depilogue.o(.text) for _double_epilogue
    ffixi.o(.text) refers (Special) to iusefp.o(.text) for __I$use$fp
    dfixi.o(.text) refers (Special) to iusefp.o(.text) for __I$use$fp
    dfixi.o(.text) refers to llushr.o(.text) for __aeabi_llsr
    entry2.o(.ARM.Collect$$$$00000001) refers to entry2.o(.ARM.Collect$$$$00002712) for __lit__00000000
    entry2.o(.ARM.Collect$$$$00002712) refers to startup_mspm0l130x_uvision.o(STACK) for __initial_sp
    entry2.o(__vectab_stack_and_reset_area) refers to startup_mspm0l130x_uvision.o(STACK) for __initial_sp
    entry2.o(__vectab_stack_and_reset_area) refers to entry.o(.ARM.Collect$$$$00000000) for __main
    entry5.o(.ARM.Collect$$$$00000004) refers to init.o(.text) for __scatterload
    entry9a.o(.ARM.Collect$$$$0000000B) refers to main.o(.text.main) for main
    entry9b.o(.ARM.Collect$$$$0000000C) refers to main.o(.text.main) for main
    idiv_div0.o(.text) refers to uidiv_div0.o(.text) for __aeabi_uidivmod
    uldiv.o(.text) refers to llushr.o(.text) for __aeabi_llsr
    uldiv.o(.text) refers to llshl.o(.text) for __aeabi_llsl
    fepilogue.o(.text) refers (Special) to iusefp.o(.text) for __I$use$fp
    depilogue.o(.text) refers (Special) to iusefp.o(.text) for __I$use$fp
    depilogue.o(.text) refers to depilogue.o(i.__ARM_clz) for __ARM_clz
    depilogue.o(.text) refers to llshl.o(.text) for __aeabi_llsl
    depilogue.o(.text) refers to llushr.o(.text) for __aeabi_llsr
    dfixul.o(.text) refers (Special) to iusefp.o(.text) for __I$use$fp
    dfixul.o(.text) refers to llushr.o(.text) for __aeabi_llsr
    dfixul.o(.text) refers to llshl.o(.text) for __aeabi_llsl
    cdrcmple.o(.text) refers (Special) to iusefp.o(.text) for __I$use$fp
    init.o(.text) refers to entry5.o(.ARM.Collect$$$$00000004) for __main_after_scatterload
    depilogue.o(i.__ARM_clz) refers (Special) to iusefp.o(.text) for __I$use$fp


==============================================================================

Removing Unused input sections from the image.

    Removing main.o(.text), (0 bytes).
    Removing main.o(.ARM.exidx.text.fputc), (8 bytes).
    Removing main.o(.ARM.exidx.text.DL_UART_isBusy), (8 bytes).
    Removing main.o(.ARM.exidx.text.DL_UART_transmitData), (8 bytes).
    Removing main.o(.ARM.exidx.text.CalculateNormalizedValue), (8 bytes).
    Removing main.o(.ARM.exidx.text.main), (8 bytes).
    Removing main.o(.ARM.exidx.text.DL_DMA_setSrcAddr), (8 bytes).
    Removing main.o(.ARM.exidx.text.DL_DMA_setDestAddr), (8 bytes).
    Removing main.o(.ARM.exidx.text.DL_DMA_enableChannel), (8 bytes).
    Removing main.o(.ARM.exidx.text.DL_ADC12_startConversion), (8 bytes).
    Removing main.o(.ARM.exidx.text.__NVIC_EnableIRQ), (8 bytes).
    Removing main.o(.ARM.exidx.text.DL_Timer_startCounter), (8 bytes).
    Removing main.o(.bss.Anolog), (16 bytes).
    Removing main.o(.rodata.cst16), (16 bytes).
    Removing main.o(.ARM.use_no_argv), (4 bytes).
    Removing startup_mspm0l130x_uvision.o(HEAP), (0 bytes).
    Removing ti_msp_dl_config.o(.text), (0 bytes).
    Removing ti_msp_dl_config.o(.ARM.exidx.text.SYSCFG_DL_init), (8 bytes).
    Removing ti_msp_dl_config.o(.ARM.exidx.text.SYSCFG_DL_initPower), (8 bytes).
    Removing ti_msp_dl_config.o(.ARM.exidx.text.SYSCFG_DL_GPIO_init), (8 bytes).
    Removing ti_msp_dl_config.o(.ARM.exidx.text.SYSCFG_DL_SYSCTL_init), (8 bytes).
    Removing ti_msp_dl_config.o(.ARM.exidx.text.SYSCFG_DL_TIMER_0_init), (8 bytes).
    Removing ti_msp_dl_config.o(.ARM.exidx.text.SYSCFG_DL_UART_0_init), (8 bytes).
    Removing ti_msp_dl_config.o(.ARM.exidx.text.SYSCFG_DL_ADC_VOLTAGE_init), (8 bytes).
    Removing ti_msp_dl_config.o(.ARM.exidx.text.SYSCFG_DL_DMA_init), (8 bytes).
    Removing ti_msp_dl_config.o(.ARM.exidx.text.SYSCFG_DL_SYSTICK_init), (8 bytes).
    Removing ti_msp_dl_config.o(.ARM.exidx.text.DL_GPIO_reset), (8 bytes).
    Removing ti_msp_dl_config.o(.ARM.exidx.text.DL_Timer_reset), (8 bytes).
    Removing ti_msp_dl_config.o(.ARM.exidx.text.DL_UART_reset), (8 bytes).
    Removing ti_msp_dl_config.o(.ARM.exidx.text.DL_ADC12_reset), (8 bytes).
    Removing ti_msp_dl_config.o(.ARM.exidx.text.DL_GPIO_enablePower), (8 bytes).
    Removing ti_msp_dl_config.o(.ARM.exidx.text.DL_Timer_enablePower), (8 bytes).
    Removing ti_msp_dl_config.o(.ARM.exidx.text.DL_UART_enablePower), (8 bytes).
    Removing ti_msp_dl_config.o(.ARM.exidx.text.DL_ADC12_enablePower), (8 bytes).
    Removing ti_msp_dl_config.o(.ARM.exidx.text.DL_GPIO_initPeripheralOutputFunction), (8 bytes).
    Removing ti_msp_dl_config.o(.ARM.exidx.text.DL_GPIO_initPeripheralInputFunction), (8 bytes).
    Removing ti_msp_dl_config.o(.ARM.exidx.text.DL_GPIO_initDigitalOutput), (8 bytes).
    Removing ti_msp_dl_config.o(.ARM.exidx.text.DL_GPIO_initDigitalInputFeatures), (8 bytes).
    Removing ti_msp_dl_config.o(.ARM.exidx.text.DL_GPIO_clearPins), (8 bytes).
    Removing ti_msp_dl_config.o(.ARM.exidx.text.DL_GPIO_enableOutput), (8 bytes).
    Removing ti_msp_dl_config.o(.ARM.exidx.text.DL_GPIO_setUpperPinsPolarity), (8 bytes).
    Removing ti_msp_dl_config.o(.ARM.exidx.text.DL_GPIO_clearInterruptStatus), (8 bytes).
    Removing ti_msp_dl_config.o(.ARM.exidx.text.DL_GPIO_enableInterrupt), (8 bytes).
    Removing ti_msp_dl_config.o(.ARM.exidx.text.DL_SYSCTL_setBORThreshold), (8 bytes).
    Removing ti_msp_dl_config.o(.ARM.exidx.text.DL_SYSCTL_setSYSOSCFreq), (8 bytes).
    Removing ti_msp_dl_config.o(.ARM.exidx.text.DL_SYSCTL_enableMFPCLK), (8 bytes).
    Removing ti_msp_dl_config.o(.ARM.exidx.text.__NVIC_SetPriority), (8 bytes).
    Removing ti_msp_dl_config.o(.ARM.exidx.text.DL_Timer_enableInterrupt), (8 bytes).
    Removing ti_msp_dl_config.o(.ARM.exidx.text.DL_Timer_enableClock), (8 bytes).
    Removing ti_msp_dl_config.o(.ARM.exidx.text.DL_UART_setOversampling), (8 bytes).
    Removing ti_msp_dl_config.o(.ARM.exidx.text.DL_UART_setBaudRateDivisor), (8 bytes).
    Removing ti_msp_dl_config.o(.ARM.exidx.text.DL_UART_enable), (8 bytes).
    Removing ti_msp_dl_config.o(.ARM.exidx.text.DL_ADC12_initSingleSample), (8 bytes).
    Removing ti_msp_dl_config.o(.ARM.exidx.text.DL_ADC12_configConversionMem), (8 bytes).
    Removing ti_msp_dl_config.o(.ARM.exidx.text.DL_ADC12_setSampleTime0), (8 bytes).
    Removing ti_msp_dl_config.o(.ARM.exidx.text.DL_ADC12_enableDMA), (8 bytes).
    Removing ti_msp_dl_config.o(.ARM.exidx.text.DL_ADC12_setDMASamplesCnt), (8 bytes).
    Removing ti_msp_dl_config.o(.ARM.exidx.text.DL_ADC12_enableDMATrigger), (8 bytes).
    Removing ti_msp_dl_config.o(.ARM.exidx.text.DL_ADC12_enableConversions), (8 bytes).
    Removing ti_msp_dl_config.o(.ARM.exidx.text.SYSCFG_DL_DMA_CH0_init), (8 bytes).
    Removing ti_msp_dl_config.o(.ARM.exidx.text.DL_DMA_setTransferSize), (8 bytes).
    Removing ti_msp_dl_config.o(.ARM.exidx.text.SysTick_Config), (8 bytes).
    Removing ti_msp_dl_config.o(.ARM.exidx.text.DL_Common_updateReg), (8 bytes).
    Removing adc.o(.text), (0 bytes).
    Removing adc.o(.ARM.exidx.text.adc_getValue), (8 bytes).
    Removing delay.o(.text), (0 bytes).
    Removing delay.o(.ARM.exidx.text.SysTick_Handler), (8 bytes).
    Removing delay.o(.ARM.exidx.text.Tick_SysTickCallback), (8 bytes).
    Removing delay.o(.ARM.exidx.text.delay_us), (8 bytes).
    Removing delay.o(.ARM.exidx.text.Tick_delay), (8 bytes).
    Removing no_mcu_ganv_grayscale_sensor.o(.text), (0 bytes).
    Removing no_mcu_ganv_grayscale_sensor.o(.ARM.exidx.text.Get_Analog_value), (8 bytes).
    Removing no_mcu_ganv_grayscale_sensor.o(.ARM.exidx.text.DL_GPIO_setPins), (8 bytes).
    Removing no_mcu_ganv_grayscale_sensor.o(.ARM.exidx.text.DL_GPIO_clearPins), (8 bytes).
    Removing no_mcu_ganv_grayscale_sensor.o(.ARM.exidx.text.convertAnalogToDigital), (8 bytes).
    Removing no_mcu_ganv_grayscale_sensor.o(.ARM.exidx.text.normalizeAnalogValues), (8 bytes).
    Removing no_mcu_ganv_grayscale_sensor.o(.ARM.exidx.text.No_MCU_Ganv_Sensor_Init_Frist), (8 bytes).
    Removing no_mcu_ganv_grayscale_sensor.o(.ARM.exidx.text.No_MCU_Ganv_Sensor_Init), (8 bytes).
    Removing no_mcu_ganv_grayscale_sensor.o(.ARM.exidx.text.No_Mcu_Ganv_Sensor_Task_Without_tick), (8 bytes).
    Removing no_mcu_ganv_grayscale_sensor.o(.text.No_Mcu_Ganv_Sensor_Task_With_tick), (92 bytes).
    Removing no_mcu_ganv_grayscale_sensor.o(.ARM.exidx.text.No_Mcu_Ganv_Sensor_Task_With_tick), (8 bytes).
    Removing no_mcu_ganv_grayscale_sensor.o(.text.Task_tick), (18 bytes).
    Removing no_mcu_ganv_grayscale_sensor.o(.ARM.exidx.text.Task_tick), (8 bytes).
    Removing no_mcu_ganv_grayscale_sensor.o(.ARM.exidx.text.Get_Digtal_For_User), (8 bytes).
    Removing no_mcu_ganv_grayscale_sensor.o(.ARM.exidx.text.Get_Normalize_For_User), (8 bytes).
    Removing no_mcu_ganv_grayscale_sensor.o(.text.Get_Anolog_Value), (54 bytes).
    Removing no_mcu_ganv_grayscale_sensor.o(.ARM.exidx.text.Get_Anolog_Value), (8 bytes).
    Removing key.o(.text), (0 bytes).
    Removing key.o(.ARM.exidx.text.GROUP1_IRQHandler), (8 bytes).
    Removing key.o(.ARM.exidx.text.DL_GPIO_getPendingInterrupt), (8 bytes).
    Removing key.o(.ARM.exidx.text.DL_GPIO_readPins), (8 bytes).
    Removing pid.o(.text), (0 bytes).
    Removing pid.o(.ARM.exidx.text.Pid_Yaw), (8 bytes).
    Removing l298n.o(.text), (0 bytes).
    Removing l298n.o(.ARM.exidx.text.Motor_SetDuty_A), (8 bytes).
    Removing l298n.o(.ARM.exidx.text.Motor_SetDuty_B), (8 bytes).
    Removing l298n.o(.ARM.exidx.text.Motor_UpdatePWM_A), (8 bytes).
    Removing l298n.o(.ARM.exidx.text.DL_GPIO_clearPins), (8 bytes).
    Removing l298n.o(.ARM.exidx.text.DL_GPIO_setPins), (8 bytes).
    Removing l298n.o(.ARM.exidx.text.TIMG0_IRQHandler), (8 bytes).
    Removing l298n.o(.ARM.exidx.text.Motor_UpdatePWM_B), (8 bytes).
    Removing l298n.o(.ARM.exidx.text.Motor_Control), (8 bytes).
    Removing retarget_io.o(.text), (0 bytes).
    Removing retarget_io.o(.text.fputc), (72 bytes).
    Removing retarget_io.o(.ARM.exidx.text.fputc), (8 bytes).
    Removing retarget_io.o(.text.stdout_putchar), (12 bytes).
    Removing retarget_io.o(.ARM.exidx.text.stdout_putchar), (8 bytes).
    Removing retarget_io.o(.text.stderr_putchar), (12 bytes).
    Removing retarget_io.o(.ARM.exidx.text.stderr_putchar), (8 bytes).
    Removing retarget_io.o(.text.fgetc), (92 bytes).
    Removing retarget_io.o(.ARM.exidx.text.fgetc), (8 bytes).
    Removing retarget_io.o(.text.stdin_getchar), (16 bytes).
    Removing retarget_io.o(.ARM.exidx.text.stdin_getchar), (8 bytes).
    Removing retarget_io.o(.text.__backspace), (72 bytes).
    Removing retarget_io.o(.ARM.exidx.text.__backspace), (8 bytes).
    Removing retarget_io.o(.text.__aeabi_assert), (148 bytes).
    Removing retarget_io.o(.ARM.exidx.text.__aeabi_assert), (8 bytes).
    Removing retarget_io.o(.text.abort), (4 bytes).
    Removing retarget_io.o(.ARM.exidx.text.abort), (8 bytes).
    Removing retarget_io.o(.bss.getchar_undo), (4 bytes).
    Removing retarget_io.o(.data.getchar_ch), (4 bytes).
    Removing retarget_io.o(.rodata.str1.1), (39 bytes).
    Removing dl_adc12.o(.text), (0 bytes).
    Removing dl_adc12.o(.ARM.exidx.text.DL_ADC12_setClockConfig), (8 bytes).
    Removing dl_adc12.o(.text.DL_ADC12_getClockConfig), (40 bytes).
    Removing dl_adc12.o(.ARM.exidx.text.DL_ADC12_getClockConfig), (8 bytes).
    Removing dl_common.o(.text), (0 bytes).
    Removing dl_common.o(.ARM.exidx.text.DL_Common_delayCycles), (8 bytes).
    Removing dl_dma.o(.text), (0 bytes).
    Removing dl_dma.o(.ARM.exidx.text.DL_DMA_initChannel), (8 bytes).
    Removing dl_timer.o(.text), (0 bytes).
    Removing dl_timer.o(.ARM.exidx.text.DL_Timer_setClockConfig), (8 bytes).
    Removing dl_timer.o(.text.DL_Timer_getClockConfig), (28 bytes).
    Removing dl_timer.o(.ARM.exidx.text.DL_Timer_getClockConfig), (8 bytes).
    Removing dl_timer.o(.ARM.exidx.text.DL_Timer_initTimerMode), (8 bytes).
    Removing dl_timer.o(.text.DL_Timer_setCaptureCompareValue), (16 bytes).
    Removing dl_timer.o(.ARM.exidx.text.DL_Timer_setCaptureCompareValue), (8 bytes).
    Removing dl_timer.o(.text.DL_Timer_setCaptureCompareCtl), (40 bytes).
    Removing dl_timer.o(.ARM.exidx.text.DL_Timer_setCaptureCompareCtl), (8 bytes).
    Removing dl_timer.o(.text.DL_Timer_initCaptureMode), (260 bytes).
    Removing dl_timer.o(.ARM.exidx.text.DL_Timer_initCaptureMode), (8 bytes).
    Removing dl_timer.o(.text.DL_Timer_setCaptureCompareInput), (26 bytes).
    Removing dl_timer.o(.ARM.exidx.text.DL_Timer_setCaptureCompareInput), (8 bytes).
    Removing dl_timer.o(.text.DL_Timer_initCaptureTriggerMode), (124 bytes).
    Removing dl_timer.o(.ARM.exidx.text.DL_Timer_initCaptureTriggerMode), (8 bytes).
    Removing dl_timer.o(.text.DL_Timer_initCaptureCombinedMode), (232 bytes).
    Removing dl_timer.o(.ARM.exidx.text.DL_Timer_initCaptureCombinedMode), (8 bytes).
    Removing dl_timer.o(.text.DL_Timer_initCompareMode), (168 bytes).
    Removing dl_timer.o(.ARM.exidx.text.DL_Timer_initCompareMode), (8 bytes).
    Removing dl_timer.o(.text.DL_Timer_initCompareTriggerMode), (112 bytes).
    Removing dl_timer.o(.ARM.exidx.text.DL_Timer_initCompareTriggerMode), (8 bytes).
    Removing dl_timer.o(.text.DL_Timer_initPWMMode), (200 bytes).
    Removing dl_timer.o(.ARM.exidx.text.DL_Timer_initPWMMode), (8 bytes).
    Removing dl_timer.o(.text.DL_Timer_setCaptureCompareAction), (36 bytes).
    Removing dl_timer.o(.ARM.exidx.text.DL_Timer_setCaptureCompareAction), (8 bytes).
    Removing dl_timer.o(.text.DL_Timer_setCaptureCompareOutCtl), (24 bytes).
    Removing dl_timer.o(.ARM.exidx.text.DL_Timer_setCaptureCompareOutCtl), (8 bytes).
    Removing dl_timer.o(.text.DL_Timer_getCaptureCompareValue), (16 bytes).
    Removing dl_timer.o(.ARM.exidx.text.DL_Timer_getCaptureCompareValue), (8 bytes).
    Removing dl_timer.o(.text.DL_Timer_getCaptureCompareCtl), (24 bytes).
    Removing dl_timer.o(.ARM.exidx.text.DL_Timer_getCaptureCompareCtl), (8 bytes).
    Removing dl_timer.o(.text.DL_Timer_enableSuppressionOfCompEvent), (24 bytes).
    Removing dl_timer.o(.ARM.exidx.text.DL_Timer_enableSuppressionOfCompEvent), (8 bytes).
    Removing dl_timer.o(.text.DL_Timer_disableSuppressionOfCompEvent), (24 bytes).
    Removing dl_timer.o(.ARM.exidx.text.DL_Timer_disableSuppressionOfCompEvent), (8 bytes).
    Removing dl_timer.o(.text.DL_Timer_setCaptCompUpdateMethod), (28 bytes).
    Removing dl_timer.o(.ARM.exidx.text.DL_Timer_setCaptCompUpdateMethod), (8 bytes).
    Removing dl_timer.o(.text.DL_Timer_getCaptCompUpdateMethod), (20 bytes).
    Removing dl_timer.o(.ARM.exidx.text.DL_Timer_getCaptCompUpdateMethod), (8 bytes).
    Removing dl_timer.o(.text.DL_Timer_getCaptureCompareOutCtl), (16 bytes).
    Removing dl_timer.o(.ARM.exidx.text.DL_Timer_getCaptureCompareOutCtl), (8 bytes).
    Removing dl_timer.o(.text.DL_Timer_getCaptureCompareAction), (24 bytes).
    Removing dl_timer.o(.ARM.exidx.text.DL_Timer_getCaptureCompareAction), (8 bytes).
    Removing dl_timer.o(.text.DL_Timer_overrideCCPOut), (32 bytes).
    Removing dl_timer.o(.ARM.exidx.text.DL_Timer_overrideCCPOut), (8 bytes).
    Removing dl_timer.o(.text.DL_Timer_getCaptureCompareInput), (16 bytes).
    Removing dl_timer.o(.ARM.exidx.text.DL_Timer_getCaptureCompareInput), (8 bytes).
    Removing dl_timer.o(.text.DL_Timer_setCaptureCompareInputFilter), (28 bytes).
    Removing dl_timer.o(.ARM.exidx.text.DL_Timer_setCaptureCompareInputFilter), (8 bytes).
    Removing dl_timer.o(.text.DL_Timer_getCaptureCompareInputFilter), (18 bytes).
    Removing dl_timer.o(.ARM.exidx.text.DL_Timer_getCaptureCompareInputFilter), (8 bytes).
    Removing dl_timer.o(.text.DL_Timer_enableCaptureCompareInputFilter), (20 bytes).
    Removing dl_timer.o(.ARM.exidx.text.DL_Timer_enableCaptureCompareInputFilter), (8 bytes).
    Removing dl_timer.o(.text.DL_Timer_disableCaptureCompareInputFilter), (20 bytes).
    Removing dl_timer.o(.ARM.exidx.text.DL_Timer_disableCaptureCompareInputFilter), (8 bytes).
    Removing dl_timer.o(.text.DL_Timer_isCaptureCompareInputFilterEnabled), (20 bytes).
    Removing dl_timer.o(.ARM.exidx.text.DL_Timer_isCaptureCompareInputFilterEnabled), (8 bytes).
    Removing dl_timer.o(.text.DL_Timer_saveConfiguration), (192 bytes).
    Removing dl_timer.o(.ARM.exidx.text.DL_Timer_saveConfiguration), (8 bytes).
    Removing dl_timer.o(.text.DL_Timer_restoreConfiguration), (196 bytes).
    Removing dl_timer.o(.ARM.exidx.text.DL_Timer_restoreConfiguration), (8 bytes).
    Removing dl_timer.o(.text.DL_Timer_configQEIHallInputMode), (32 bytes).
    Removing dl_timer.o(.ARM.exidx.text.DL_Timer_configQEIHallInputMode), (8 bytes).
    Removing dl_timer.o(.rodata..Lswitch.table.DL_Timer_initCompareMode), (12 bytes).
    Removing dl_uart.o(.text), (0 bytes).
    Removing dl_uart.o(.ARM.exidx.text.DL_UART_init), (8 bytes).
    Removing dl_uart.o(.ARM.exidx.text.DL_UART_setClockConfig), (8 bytes).
    Removing dl_uart.o(.text.DL_UART_getClockConfig), (16 bytes).
    Removing dl_uart.o(.ARM.exidx.text.DL_UART_getClockConfig), (8 bytes).
    Removing dl_uart.o(.text.DL_UART_configBaudRate), (140 bytes).
    Removing dl_uart.o(.ARM.exidx.text.DL_UART_configBaudRate), (8 bytes).
    Removing dl_uart.o(.text.DL_UART_configIrDAMode), (60 bytes).
    Removing dl_uart.o(.ARM.exidx.text.DL_UART_configIrDAMode), (8 bytes).
    Removing dl_uart.o(.text.DL_UART_setIrDAPulseLength), (42 bytes).
    Removing dl_uart.o(.ARM.exidx.text.DL_UART_setIrDAPulseLength), (8 bytes).
    Removing dl_uart.o(.text.DL_UART_receiveDataBlocking), (20 bytes).
    Removing dl_uart.o(.ARM.exidx.text.DL_UART_receiveDataBlocking), (8 bytes).
    Removing dl_uart.o(.text.DL_UART_transmitDataBlocking), (20 bytes).
    Removing dl_uart.o(.ARM.exidx.text.DL_UART_transmitDataBlocking), (8 bytes).
    Removing dl_uart.o(.text.DL_UART_receiveDataCheck), (28 bytes).
    Removing dl_uart.o(.ARM.exidx.text.DL_UART_receiveDataCheck), (8 bytes).
    Removing dl_uart.o(.text.DL_UART_transmitDataCheck), (24 bytes).
    Removing dl_uart.o(.ARM.exidx.text.DL_UART_transmitDataCheck), (8 bytes).
    Removing dl_uart.o(.text.DL_UART_drainRXFIFO), (40 bytes).
    Removing dl_uart.o(.ARM.exidx.text.DL_UART_drainRXFIFO), (8 bytes).
    Removing dl_uart.o(.text.DL_UART_fillTXFIFO), (40 bytes).
    Removing dl_uart.o(.ARM.exidx.text.DL_UART_fillTXFIFO), (8 bytes).
    Removing dl_uart.o(.text.DL_UART_Main_saveConfiguration), (88 bytes).
    Removing dl_uart.o(.ARM.exidx.text.DL_UART_Main_saveConfiguration), (8 bytes).
    Removing dl_uart.o(.text.DL_UART_Main_restoreConfiguration), (120 bytes).
    Removing dl_uart.o(.ARM.exidx.text.DL_UART_Main_restoreConfiguration), (8 bytes).
    Removing dl_uart.o(.text.DL_UART_Extend_saveConfiguration), (104 bytes).
    Removing dl_uart.o(.ARM.exidx.text.DL_UART_Extend_saveConfiguration), (8 bytes).
    Removing dl_uart.o(.text.DL_UART_Extend_restoreConfiguration), (132 bytes).
    Removing dl_uart.o(.ARM.exidx.text.DL_UART_Extend_restoreConfiguration), (8 bytes).

225 unused section(s) (total 4793 bytes) removed from the image.

==============================================================================

Image Symbol Table

    Local Symbols

    Symbol Name                              Value     Ov Type        Size  Object(Section)

    ../clib/division.s                       0x00000000   Number         0  aeabi_sdivfast.o ABSOLUTE
    ../clib/division.s                       0x00000000   Number         0  aeabi_sdivfast_div0.o ABSOLUTE
    ../clib/microlib/division.c              0x00000000   Number         0  uidiv.o ABSOLUTE
    ../clib/microlib/division.c              0x00000000   Number         0  idiv.o ABSOLUTE
    ../clib/microlib/division.c              0x00000000   Number         0  uidiv_div0.o ABSOLUTE
    ../clib/microlib/division.c              0x00000000   Number         0  idiv_div0.o ABSOLUTE
    ../clib/microlib/division.c              0x00000000   Number         0  idiv0.o ABSOLUTE
    ../clib/microlib/division.c              0x00000000   Number         0  uldiv.o ABSOLUTE
    ../clib/microlib/init/entry.s            0x00000000   Number         0  entry.o ABSOLUTE
    ../clib/microlib/init/entry.s            0x00000000   Number         0  entry2.o ABSOLUTE
    ../clib/microlib/init/entry.s            0x00000000   Number         0  entry5.o ABSOLUTE
    ../clib/microlib/init/entry.s            0x00000000   Number         0  entry7a.o ABSOLUTE
    ../clib/microlib/init/entry.s            0x00000000   Number         0  entry7b.o ABSOLUTE
    ../clib/microlib/init/entry.s            0x00000000   Number         0  entry8a.o ABSOLUTE
    ../clib/microlib/init/entry.s            0x00000000   Number         0  entry8b.o ABSOLUTE
    ../clib/microlib/init/entry.s            0x00000000   Number         0  entry9a.o ABSOLUTE
    ../clib/microlib/init/entry.s            0x00000000   Number         0  entry9b.o ABSOLUTE
    ../clib/microlib/init/entry.s            0x00000000   Number         0  entry10a.o ABSOLUTE
    ../clib/microlib/init/entry.s            0x00000000   Number         0  entry10b.o ABSOLUTE
    ../clib/microlib/init/entry.s            0x00000000   Number         0  entry11a.o ABSOLUTE
    ../clib/microlib/init/entry.s            0x00000000   Number         0  entry11b.o ABSOLUTE
    ../clib/microlib/longlong.c              0x00000000   Number         0  llshl.o ABSOLUTE
    ../clib/microlib/longlong.c              0x00000000   Number         0  llushr.o ABSOLUTE
    ../clib/microlib/longlong.c              0x00000000   Number         0  llsshr.o ABSOLUTE
    ../clib/microlib/printf/printf.c         0x00000000   Number         0  printfa.o ABSOLUTE
    ../clib/microlib/stdio/fputs.c           0x00000000   Number         0  fputs.o ABSOLUTE
    ../clib/microlib/stdio/fputs.c           0x00000000   Number         0  fputs_e.o ABSOLUTE
    ../clib/microlib/stdio/streams.c         0x00000000   Number         0  stdin.o ABSOLUTE
    ../clib/microlib/stdio/streams.c         0x00000000   Number         0  stdout.o ABSOLUTE
    ../clib/microlib/stdio/streams.c         0x00000000   Number         0  stderr.o ABSOLUTE
    ../clib/microlib/string/memcpy.c         0x00000000   Number         0  memcpya.o ABSOLUTE
    ../clib/microlib/string/memcpy.c         0x00000000   Number         0  memcpyb.o ABSOLUTE
    ../clib/microlib/string/memset.c         0x00000000   Number         0  memseta.o ABSOLUTE
    ../clib/microlib/stubs.s                 0x00000000   Number         0  iusefp.o ABSOLUTE
    ../fplib/microlib/fpadd.c                0x00000000   Number         0  fadd.o ABSOLUTE
    ../fplib/microlib/fpadd.c                0x00000000   Number         0  dadd.o ABSOLUTE
    ../fplib/microlib/fpcmp.c                0x00000000   Number         0  dcmple.o ABSOLUTE
    ../fplib/microlib/fpdiv.c                0x00000000   Number         0  ddiv.o ABSOLUTE
    ../fplib/microlib/fpepilogue.c           0x00000000   Number         0  fepilogue.o ABSOLUTE
    ../fplib/microlib/fpepilogue.c           0x00000000   Number         0  depilogue.o ABSOLUTE
    ../fplib/microlib/fpfix.c                0x00000000   Number         0  ffixi.o ABSOLUTE
    ../fplib/microlib/fpfix.c                0x00000000   Number         0  dfixi.o ABSOLUTE
    ../fplib/microlib/fpfix.c                0x00000000   Number         0  dfixul.o ABSOLUTE
    ../fplib/microlib/fpflt.c                0x00000000   Number         0  fflti.o ABSOLUTE
    ../fplib/microlib/fpflt.c                0x00000000   Number         0  dflti.o ABSOLUTE
    ../fplib/microlib/fpflt.c                0x00000000   Number         0  dfltui.o ABSOLUTE
    ../fplib/microlib/fpmul.c                0x00000000   Number         0  dmul.o ABSOLUTE
    L298N.c                                  0x00000000   Number         0  l298n.o ABSOLUTE
    No_Mcu_Ganv_Grayscale_Sensor.c           0x00000000   Number         0  no_mcu_ganv_grayscale_sensor.o ABSOLUTE
    PID.c                                    0x00000000   Number         0  pid.o ABSOLUTE
    adc.c                                    0x00000000   Number         0  adc.o ABSOLUTE
    cdrcmple.s                               0x00000000   Number         0  cdrcmple.o ABSOLUTE
    dc.s                                     0x00000000   Number         0  dc.o ABSOLUTE
    delay.c                                  0x00000000   Number         0  delay.o ABSOLUTE
    dl_adc12.c                               0x00000000   Number         0  dl_adc12.o ABSOLUTE
    dl_common.c                              0x00000000   Number         0  dl_common.o ABSOLUTE
    dl_dma.c                                 0x00000000   Number         0  dl_dma.o ABSOLUTE
    dl_timer.c                               0x00000000   Number         0  dl_timer.o ABSOLUTE
    dl_uart.c                                0x00000000   Number         0  dl_uart.o ABSOLUTE
    handlers.s                               0x00000000   Number         0  handlers.o ABSOLUTE
    init.s                                   0x00000000   Number         0  init.o ABSOLUTE
    key.c                                    0x00000000   Number         0  key.o ABSOLUTE
    main.c                                   0x00000000   Number         0  main.o ABSOLUTE
    retarget_io.c                            0x00000000   Number         0  retarget_io.o ABSOLUTE
    startup_mspm0l130x_uvision.s             0x00000000   Number         0  startup_mspm0l130x_uvision.o ABSOLUTE
    ti_msp_dl_config.c                       0x00000000   Number         0  ti_msp_dl_config.o ABSOLUTE
    RESET                                    0x00000000   Section      192  startup_mspm0l130x_uvision.o(RESET)
    .ARM.Collect$$$$00000000                 0x000000c0   Section        0  entry.o(.ARM.Collect$$$$00000000)
    .ARM.Collect$$$$00000001                 0x000000c0   Section        4  entry2.o(.ARM.Collect$$$$00000001)
    .ARM.Collect$$$$00000004                 0x000000c4   Section        4  entry5.o(.ARM.Collect$$$$00000004)
    .ARM.Collect$$$$00000008                 0x000000c8   Section        0  entry7b.o(.ARM.Collect$$$$00000008)
    .ARM.Collect$$$$0000000A                 0x000000c8   Section        0  entry8b.o(.ARM.Collect$$$$0000000A)
    .ARM.Collect$$$$0000000B                 0x000000c8   Section        8  entry9a.o(.ARM.Collect$$$$0000000B)
    __lit__00000000                          0x000000d0   Data           4  entry2.o(.ARM.Collect$$$$00002712)
    .ARM.Collect$$$$0000000D                 0x000000d0   Section        0  entry10a.o(.ARM.Collect$$$$0000000D)
    .ARM.Collect$$$$0000000F                 0x000000d0   Section        0  entry11a.o(.ARM.Collect$$$$0000000F)
    .ARM.Collect$$$$00002712                 0x000000d0   Section        4  entry2.o(.ARM.Collect$$$$00002712)
    .text                                    0x000000d4   Section       20  startup_mspm0l130x_uvision.o(.text)
    .text                                    0x000000e8   Section        0  memcpya.o(.text)
    .text                                    0x0000010c   Section        0  memseta.o(.text)
    .text                                    0x00000130   Section        0  fadd.o(.text)
    .text                                    0x000001e4   Section        0  dadd.o(.text)
    .text                                    0x00000348   Section        0  dmul.o(.text)
    .text                                    0x00000418   Section        0  ddiv.o(.text)
    .text                                    0x00000508   Section        0  dcmple.o(.text)
    .text                                    0x00000534   Section        0  fflti.o(.text)
    .text                                    0x0000054c   Section        0  dflti.o(.text)
    .text                                    0x00000574   Section        0  dfltui.o(.text)
    .text                                    0x00000590   Section        0  ffixi.o(.text)
    .text                                    0x000005c4   Section        0  dfixi.o(.text)
    .text                                    0x0000060c   Section        0  uidiv_div0.o(.text)
    .text                                    0x0000064c   Section        0  idiv_div0.o(.text)
    .text                                    0x0000069c   Section        0  uldiv.o(.text)
    .text                                    0x000006fc   Section        0  llshl.o(.text)
    .text                                    0x0000071c   Section        0  llushr.o(.text)
    .text                                    0x0000073e   Section        0  llsshr.o(.text)
    .text                                    0x00000764   Section        0  iusefp.o(.text)
    .text                                    0x00000764   Section        0  fepilogue.o(.text)
    .text                                    0x000007e6   Section        0  depilogue.o(.text)
    .text                                    0x000008a4   Section        0  dfixul.o(.text)
    .text                                    0x000008e4   Section       40  cdrcmple.o(.text)
    .text                                    0x00000910   Section       48  init.o(.text)
    [Anonymous Symbol]                       0x00000940   Section        0  main.o(.text.CalculateNormalizedValue)
    __arm_cp.3_0                             0x00000a10   Number         4  main.o(.text.CalculateNormalizedValue)
    __arm_cp.3_1                             0x00000a14   Number         4  main.o(.text.CalculateNormalizedValue)
    __arm_cp.3_2                             0x00000a18   Number         4  main.o(.text.CalculateNormalizedValue)
    __arm_cp.3_3                             0x00000a1c   Number         4  main.o(.text.CalculateNormalizedValue)
    DL_ADC12_configConversionMem             0x00000a21   Thumb Code    74  ti_msp_dl_config.o(.text.DL_ADC12_configConversionMem)
    [Anonymous Symbol]                       0x00000a20   Section        0  ti_msp_dl_config.o(.text.DL_ADC12_configConversionMem)
    DL_ADC12_enableConversions               0x00000a6b   Thumb Code    22  ti_msp_dl_config.o(.text.DL_ADC12_enableConversions)
    [Anonymous Symbol]                       0x00000a6a   Section        0  ti_msp_dl_config.o(.text.DL_ADC12_enableConversions)
    DL_ADC12_enableDMA                       0x00000a81   Thumb Code    24  ti_msp_dl_config.o(.text.DL_ADC12_enableDMA)
    [Anonymous Symbol]                       0x00000a80   Section        0  ti_msp_dl_config.o(.text.DL_ADC12_enableDMA)
    DL_ADC12_enableDMATrigger                0x00000a99   Thumb Code    24  ti_msp_dl_config.o(.text.DL_ADC12_enableDMATrigger)
    [Anonymous Symbol]                       0x00000a98   Section        0  ti_msp_dl_config.o(.text.DL_ADC12_enableDMATrigger)
    __arm_cp.40_0                            0x00000ab0   Number         4  ti_msp_dl_config.o(.text.DL_ADC12_enableDMATrigger)
    DL_ADC12_enablePower                     0x00000ab5   Thumb Code    20  ti_msp_dl_config.o(.text.DL_ADC12_enablePower)
    [Anonymous Symbol]                       0x00000ab4   Section        0  ti_msp_dl_config.o(.text.DL_ADC12_enablePower)
    DL_ADC12_initSingleSample                0x00000ac9   Thumb Code    60  ti_msp_dl_config.o(.text.DL_ADC12_initSingleSample)
    [Anonymous Symbol]                       0x00000ac8   Section        0  ti_msp_dl_config.o(.text.DL_ADC12_initSingleSample)
    __arm_cp.35_1                            0x00000b04   Number         4  ti_msp_dl_config.o(.text.DL_ADC12_initSingleSample)
    __arm_cp.35_3                            0x00000b08   Number         4  ti_msp_dl_config.o(.text.DL_ADC12_initSingleSample)
    DL_ADC12_reset                           0x00000b0d   Thumb Code    16  ti_msp_dl_config.o(.text.DL_ADC12_reset)
    [Anonymous Symbol]                       0x00000b0c   Section        0  ti_msp_dl_config.o(.text.DL_ADC12_reset)
    [Anonymous Symbol]                       0x00000b1c   Section        0  dl_adc12.o(.text.DL_ADC12_setClockConfig)
    __arm_cp.0_0                             0x00000b54   Number         4  dl_adc12.o(.text.DL_ADC12_setClockConfig)
    __arm_cp.0_1                             0x00000b58   Number         4  dl_adc12.o(.text.DL_ADC12_setClockConfig)
    DL_ADC12_setDMASamplesCnt                0x00000b5d   Thumb Code    40  ti_msp_dl_config.o(.text.DL_ADC12_setDMASamplesCnt)
    [Anonymous Symbol]                       0x00000b5c   Section        0  ti_msp_dl_config.o(.text.DL_ADC12_setDMASamplesCnt)
    __arm_cp.39_0                            0x00000b84   Number         4  ti_msp_dl_config.o(.text.DL_ADC12_setDMASamplesCnt)
    DL_ADC12_setSampleTime0                  0x00000b89   Thumb Code    20  ti_msp_dl_config.o(.text.DL_ADC12_setSampleTime0)
    [Anonymous Symbol]                       0x00000b88   Section        0  ti_msp_dl_config.o(.text.DL_ADC12_setSampleTime0)
    __arm_cp.37_0                            0x00000b9c   Number         4  ti_msp_dl_config.o(.text.DL_ADC12_setSampleTime0)
    DL_ADC12_startConversion                 0x00000ba1   Thumb Code    24  main.o(.text.DL_ADC12_startConversion)
    [Anonymous Symbol]                       0x00000ba0   Section        0  main.o(.text.DL_ADC12_startConversion)
    __arm_cp.8_0                             0x00000bb8   Number         4  main.o(.text.DL_ADC12_startConversion)
    [Anonymous Symbol]                       0x00000bbc   Section        0  dl_common.o(.text.DL_Common_delayCycles)
    DL_Common_updateReg                      0x00000bc7   Thumb Code    40  ti_msp_dl_config.o(.text.DL_Common_updateReg)
    [Anonymous Symbol]                       0x00000bc6   Section        0  ti_msp_dl_config.o(.text.DL_Common_updateReg)
    DL_DMA_enableChannel                     0x00000bef   Thumb Code    38  main.o(.text.DL_DMA_enableChannel)
    [Anonymous Symbol]                       0x00000bee   Section        0  main.o(.text.DL_DMA_enableChannel)
    [Anonymous Symbol]                       0x00000c14   Section        0  dl_dma.o(.text.DL_DMA_initChannel)
    __arm_cp.0_0                             0x00000c54   Number         4  dl_dma.o(.text.DL_DMA_initChannel)
    DL_DMA_setDestAddr                       0x00000c59   Thumb Code    36  main.o(.text.DL_DMA_setDestAddr)
    [Anonymous Symbol]                       0x00000c58   Section        0  main.o(.text.DL_DMA_setDestAddr)
    __arm_cp.6_0                             0x00000c7c   Number         4  main.o(.text.DL_DMA_setDestAddr)
    DL_DMA_setSrcAddr                        0x00000c81   Thumb Code    36  main.o(.text.DL_DMA_setSrcAddr)
    [Anonymous Symbol]                       0x00000c80   Section        0  main.o(.text.DL_DMA_setSrcAddr)
    __arm_cp.5_0                             0x00000ca4   Number         4  main.o(.text.DL_DMA_setSrcAddr)
    DL_DMA_setTransferSize                   0x00000ca9   Thumb Code    44  ti_msp_dl_config.o(.text.DL_DMA_setTransferSize)
    [Anonymous Symbol]                       0x00000ca8   Section        0  ti_msp_dl_config.o(.text.DL_DMA_setTransferSize)
    __arm_cp.43_0                            0x00000cd4   Number         4  ti_msp_dl_config.o(.text.DL_DMA_setTransferSize)
    DL_GPIO_clearInterruptStatus             0x00000cd9   Thumb Code    24  ti_msp_dl_config.o(.text.DL_GPIO_clearInterruptStatus)
    [Anonymous Symbol]                       0x00000cd8   Section        0  ti_msp_dl_config.o(.text.DL_GPIO_clearInterruptStatus)
    __arm_cp.24_0                            0x00000cf0   Number         4  ti_msp_dl_config.o(.text.DL_GPIO_clearInterruptStatus)
    DL_GPIO_clearPins                        0x00000cf5   Thumb Code    20  ti_msp_dl_config.o(.text.DL_GPIO_clearPins)
    [Anonymous Symbol]                       0x00000cf4   Section        0  ti_msp_dl_config.o(.text.DL_GPIO_clearPins)
    DL_GPIO_clearPins                        0x00000d09   Thumb Code    20  no_mcu_ganv_grayscale_sensor.o(.text.DL_GPIO_clearPins)
    [Anonymous Symbol]                       0x00000d08   Section        0  no_mcu_ganv_grayscale_sensor.o(.text.DL_GPIO_clearPins)
    DL_GPIO_clearPins                        0x00000d1d   Thumb Code    20  l298n.o(.text.DL_GPIO_clearPins)
    [Anonymous Symbol]                       0x00000d1c   Section        0  l298n.o(.text.DL_GPIO_clearPins)
    DL_GPIO_enableInterrupt                  0x00000d31   Thumb Code    24  ti_msp_dl_config.o(.text.DL_GPIO_enableInterrupt)
    [Anonymous Symbol]                       0x00000d30   Section        0  ti_msp_dl_config.o(.text.DL_GPIO_enableInterrupt)
    DL_GPIO_enableOutput                     0x00000d49   Thumb Code    20  ti_msp_dl_config.o(.text.DL_GPIO_enableOutput)
    [Anonymous Symbol]                       0x00000d48   Section        0  ti_msp_dl_config.o(.text.DL_GPIO_enableOutput)
    __arm_cp.22_0                            0x00000d5c   Number         4  ti_msp_dl_config.o(.text.DL_GPIO_enableOutput)
    DL_GPIO_enablePower                      0x00000d61   Thumb Code    20  ti_msp_dl_config.o(.text.DL_GPIO_enablePower)
    [Anonymous Symbol]                       0x00000d60   Section        0  ti_msp_dl_config.o(.text.DL_GPIO_enablePower)
    __arm_cp.13_0                            0x00000d74   Number         4  ti_msp_dl_config.o(.text.DL_GPIO_enablePower)
    DL_GPIO_getPendingInterrupt              0x00000d79   Thumb Code    18  key.o(.text.DL_GPIO_getPendingInterrupt)
    [Anonymous Symbol]                       0x00000d78   Section        0  key.o(.text.DL_GPIO_getPendingInterrupt)
    DL_GPIO_initDigitalInputFeatures         0x00000d8d   Thumb Code    44  ti_msp_dl_config.o(.text.DL_GPIO_initDigitalInputFeatures)
    [Anonymous Symbol]                       0x00000d8c   Section        0  ti_msp_dl_config.o(.text.DL_GPIO_initDigitalInputFeatures)
    __arm_cp.20_0                            0x00000db8   Number         4  ti_msp_dl_config.o(.text.DL_GPIO_initDigitalInputFeatures)
    DL_GPIO_initDigitalOutput                0x00000dbd   Thumb Code    20  ti_msp_dl_config.o(.text.DL_GPIO_initDigitalOutput)
    [Anonymous Symbol]                       0x00000dbc   Section        0  ti_msp_dl_config.o(.text.DL_GPIO_initDigitalOutput)
    DL_GPIO_initPeripheralInputFunction      0x00000dd1   Thumb Code    24  ti_msp_dl_config.o(.text.DL_GPIO_initPeripheralInputFunction)
    [Anonymous Symbol]                       0x00000dd0   Section        0  ti_msp_dl_config.o(.text.DL_GPIO_initPeripheralInputFunction)
    __arm_cp.18_0                            0x00000de8   Number         4  ti_msp_dl_config.o(.text.DL_GPIO_initPeripheralInputFunction)
    DL_GPIO_initPeripheralOutputFunction     0x00000ded   Thumb Code    24  ti_msp_dl_config.o(.text.DL_GPIO_initPeripheralOutputFunction)
    [Anonymous Symbol]                       0x00000dec   Section        0  ti_msp_dl_config.o(.text.DL_GPIO_initPeripheralOutputFunction)
    __arm_cp.17_0                            0x00000e04   Number         4  ti_msp_dl_config.o(.text.DL_GPIO_initPeripheralOutputFunction)
    DL_GPIO_readPins                         0x00000e09   Thumb Code    22  key.o(.text.DL_GPIO_readPins)
    [Anonymous Symbol]                       0x00000e08   Section        0  key.o(.text.DL_GPIO_readPins)
    DL_GPIO_reset                            0x00000e21   Thumb Code    16  ti_msp_dl_config.o(.text.DL_GPIO_reset)
    [Anonymous Symbol]                       0x00000e20   Section        0  ti_msp_dl_config.o(.text.DL_GPIO_reset)
    __arm_cp.9_0                             0x00000e30   Number         4  ti_msp_dl_config.o(.text.DL_GPIO_reset)
    __arm_cp.9_1                             0x00000e34   Number         4  ti_msp_dl_config.o(.text.DL_GPIO_reset)
    DL_GPIO_setPins                          0x00000e39   Thumb Code    20  no_mcu_ganv_grayscale_sensor.o(.text.DL_GPIO_setPins)
    [Anonymous Symbol]                       0x00000e38   Section        0  no_mcu_ganv_grayscale_sensor.o(.text.DL_GPIO_setPins)
    DL_GPIO_setPins                          0x00000e4d   Thumb Code    20  l298n.o(.text.DL_GPIO_setPins)
    [Anonymous Symbol]                       0x00000e4c   Section        0  l298n.o(.text.DL_GPIO_setPins)
    __arm_cp.4_0                             0x00000e60   Number         4  l298n.o(.text.DL_GPIO_setPins)
    DL_GPIO_setUpperPinsPolarity             0x00000e65   Thumb Code    24  ti_msp_dl_config.o(.text.DL_GPIO_setUpperPinsPolarity)
    [Anonymous Symbol]                       0x00000e64   Section        0  ti_msp_dl_config.o(.text.DL_GPIO_setUpperPinsPolarity)
    DL_SYSCTL_enableMFPCLK                   0x00000e7d   Thumb Code    12  ti_msp_dl_config.o(.text.DL_SYSCTL_enableMFPCLK)
    [Anonymous Symbol]                       0x00000e7c   Section        0  ti_msp_dl_config.o(.text.DL_SYSCTL_enableMFPCLK)
    __arm_cp.28_0                            0x00000e88   Number         4  ti_msp_dl_config.o(.text.DL_SYSCTL_enableMFPCLK)
    DL_SYSCTL_setBORThreshold                0x00000e8d   Thumb Code    20  ti_msp_dl_config.o(.text.DL_SYSCTL_setBORThreshold)
    [Anonymous Symbol]                       0x00000e8c   Section        0  ti_msp_dl_config.o(.text.DL_SYSCTL_setBORThreshold)
    __arm_cp.26_0                            0x00000ea0   Number         4  ti_msp_dl_config.o(.text.DL_SYSCTL_setBORThreshold)
    DL_SYSCTL_setSYSOSCFreq                  0x00000ea5   Thumb Code    24  ti_msp_dl_config.o(.text.DL_SYSCTL_setSYSOSCFreq)
    [Anonymous Symbol]                       0x00000ea4   Section        0  ti_msp_dl_config.o(.text.DL_SYSCTL_setSYSOSCFreq)
    __arm_cp.27_0                            0x00000ebc   Number         4  ti_msp_dl_config.o(.text.DL_SYSCTL_setSYSOSCFreq)
    DL_Timer_enableClock                     0x00000ec1   Thumb Code    16  ti_msp_dl_config.o(.text.DL_Timer_enableClock)
    [Anonymous Symbol]                       0x00000ec0   Section        0  ti_msp_dl_config.o(.text.DL_Timer_enableClock)
    __arm_cp.31_0                            0x00000ed0   Number         4  ti_msp_dl_config.o(.text.DL_Timer_enableClock)
    DL_Timer_enableInterrupt                 0x00000ed5   Thumb Code    24  ti_msp_dl_config.o(.text.DL_Timer_enableInterrupt)
    [Anonymous Symbol]                       0x00000ed4   Section        0  ti_msp_dl_config.o(.text.DL_Timer_enableInterrupt)
    __arm_cp.30_0                            0x00000eec   Number         4  ti_msp_dl_config.o(.text.DL_Timer_enableInterrupt)
    DL_Timer_enablePower                     0x00000ef1   Thumb Code    20  ti_msp_dl_config.o(.text.DL_Timer_enablePower)
    [Anonymous Symbol]                       0x00000ef0   Section        0  ti_msp_dl_config.o(.text.DL_Timer_enablePower)
    [Anonymous Symbol]                       0x00000f04   Section        0  dl_timer.o(.text.DL_Timer_initTimerMode)
    __arm_cp.2_0                             0x00000fe4   Number         4  dl_timer.o(.text.DL_Timer_initTimerMode)
    __arm_cp.2_2                             0x00000fe8   Number         4  dl_timer.o(.text.DL_Timer_initTimerMode)
    __arm_cp.2_3                             0x00000fec   Number         4  dl_timer.o(.text.DL_Timer_initTimerMode)
    DL_Timer_reset                           0x00000ff1   Thumb Code    16  ti_msp_dl_config.o(.text.DL_Timer_reset)
    [Anonymous Symbol]                       0x00000ff0   Section        0  ti_msp_dl_config.o(.text.DL_Timer_reset)
    [Anonymous Symbol]                       0x00001000   Section        0  dl_timer.o(.text.DL_Timer_setClockConfig)
    __arm_cp.0_0                             0x00001018   Number         4  dl_timer.o(.text.DL_Timer_setClockConfig)
    DL_Timer_startCounter                    0x0000101d   Thumb Code    20  main.o(.text.DL_Timer_startCounter)
    [Anonymous Symbol]                       0x0000101c   Section        0  main.o(.text.DL_Timer_startCounter)
    __arm_cp.10_0                            0x00001030   Number         4  main.o(.text.DL_Timer_startCounter)
    DL_UART_enable                           0x00001035   Thumb Code    22  ti_msp_dl_config.o(.text.DL_UART_enable)
    [Anonymous Symbol]                       0x00001034   Section        0  ti_msp_dl_config.o(.text.DL_UART_enable)
    DL_UART_enablePower                      0x0000104d   Thumb Code    20  ti_msp_dl_config.o(.text.DL_UART_enablePower)
    [Anonymous Symbol]                       0x0000104c   Section        0  ti_msp_dl_config.o(.text.DL_UART_enablePower)
    __arm_cp.15_0                            0x00001060   Number         4  ti_msp_dl_config.o(.text.DL_UART_enablePower)
    [Anonymous Symbol]                       0x00001064   Section        0  dl_uart.o(.text.DL_UART_init)
    __arm_cp.0_0                             0x000010a4   Number         4  dl_uart.o(.text.DL_UART_init)
    __arm_cp.0_1                             0x000010a8   Number         4  dl_uart.o(.text.DL_UART_init)
    DL_UART_isBusy                           0x000010ad   Thumb Code    20  main.o(.text.DL_UART_isBusy)
    [Anonymous Symbol]                       0x000010ac   Section        0  main.o(.text.DL_UART_isBusy)
    __arm_cp.1_0                             0x000010c0   Number         4  main.o(.text.DL_UART_isBusy)
    DL_UART_reset                            0x000010c5   Thumb Code    16  ti_msp_dl_config.o(.text.DL_UART_reset)
    [Anonymous Symbol]                       0x000010c4   Section        0  ti_msp_dl_config.o(.text.DL_UART_reset)
    __arm_cp.11_0                            0x000010d4   Number         4  ti_msp_dl_config.o(.text.DL_UART_reset)
    __arm_cp.11_1                            0x000010d8   Number         4  ti_msp_dl_config.o(.text.DL_UART_reset)
    DL_UART_setBaudRateDivisor               0x000010dd   Thumb Code    60  ti_msp_dl_config.o(.text.DL_UART_setBaudRateDivisor)
    [Anonymous Symbol]                       0x000010dc   Section        0  ti_msp_dl_config.o(.text.DL_UART_setBaudRateDivisor)
    __arm_cp.33_0                            0x00001118   Number         4  ti_msp_dl_config.o(.text.DL_UART_setBaudRateDivisor)
    __arm_cp.33_1                            0x0000111c   Number         4  ti_msp_dl_config.o(.text.DL_UART_setBaudRateDivisor)
    __arm_cp.33_2                            0x00001120   Number         4  ti_msp_dl_config.o(.text.DL_UART_setBaudRateDivisor)
    __arm_cp.33_3                            0x00001124   Number         4  ti_msp_dl_config.o(.text.DL_UART_setBaudRateDivisor)
    [Anonymous Symbol]                       0x00001128   Section        0  dl_uart.o(.text.DL_UART_setClockConfig)
    DL_UART_setOversampling                  0x0000113b   Thumb Code    30  ti_msp_dl_config.o(.text.DL_UART_setOversampling)
    [Anonymous Symbol]                       0x0000113a   Section        0  ti_msp_dl_config.o(.text.DL_UART_setOversampling)
    DL_UART_transmitData                     0x00001159   Thumb Code    22  main.o(.text.DL_UART_transmitData)
    [Anonymous Symbol]                       0x00001158   Section        0  main.o(.text.DL_UART_transmitData)
    [Anonymous Symbol]                       0x00001170   Section        0  key.o(.text.GROUP1_IRQHandler)
    __arm_cp.0_1                             0x000011cc   Number         4  key.o(.text.GROUP1_IRQHandler)
    __arm_cp.0_2                             0x000011d0   Number         4  key.o(.text.GROUP1_IRQHandler)
    __arm_cp.0_3                             0x000011d4   Number         4  key.o(.text.GROUP1_IRQHandler)
    __arm_cp.0_4                             0x000011d8   Number         4  key.o(.text.GROUP1_IRQHandler)
    [Anonymous Symbol]                       0x000011dc   Section        0  no_mcu_ganv_grayscale_sensor.o(.text.Get_Analog_value)
    [Anonymous Symbol]                       0x00001294   Section        0  no_mcu_ganv_grayscale_sensor.o(.text.Get_Digtal_For_User)
    [Anonymous Symbol]                       0x000012a2   Section        0  no_mcu_ganv_grayscale_sensor.o(.text.Get_Normalize_For_User)
    [Anonymous Symbol]                       0x000012dc   Section        0  l298n.o(.text.Motor_Control)
    __arm_cp.7_0                             0x00001404   Number         4  l298n.o(.text.Motor_Control)
    __arm_cp.7_1                             0x00001408   Number         4  l298n.o(.text.Motor_Control)
    __arm_cp.7_2                             0x0000140c   Number         4  l298n.o(.text.Motor_Control)
    __arm_cp.7_3                             0x00001410   Number         4  l298n.o(.text.Motor_Control)
    __arm_cp.7_4                             0x00001414   Number         4  l298n.o(.text.Motor_Control)
    __arm_cp.7_5                             0x00001418   Number         4  l298n.o(.text.Motor_Control)
    __arm_cp.7_6                             0x0000141c   Number         4  l298n.o(.text.Motor_Control)
    __arm_cp.7_7                             0x00001420   Number         4  l298n.o(.text.Motor_Control)
    __arm_cp.7_8                             0x00001424   Number         4  l298n.o(.text.Motor_Control)
    __arm_cp.7_9                             0x00001428   Number         4  l298n.o(.text.Motor_Control)
    [Anonymous Symbol]                       0x0000142c   Section        0  l298n.o(.text.Motor_SetDuty_A)
    [Anonymous Symbol]                       0x00001464   Section        0  l298n.o(.text.Motor_SetDuty_B)
    [Anonymous Symbol]                       0x0000149c   Section        0  l298n.o(.text.Motor_UpdatePWM_A)
    __arm_cp.2_0                             0x0000153c   Number         4  l298n.o(.text.Motor_UpdatePWM_A)
    __arm_cp.2_1                             0x00001540   Number         4  l298n.o(.text.Motor_UpdatePWM_A)
    __arm_cp.2_2                             0x00001544   Number         4  l298n.o(.text.Motor_UpdatePWM_A)
    [Anonymous Symbol]                       0x00001548   Section        0  l298n.o(.text.Motor_UpdatePWM_B)
    __arm_cp.6_0                             0x00001600   Number         4  l298n.o(.text.Motor_UpdatePWM_B)
    __arm_cp.6_1                             0x00001604   Number         4  l298n.o(.text.Motor_UpdatePWM_B)
    __arm_cp.6_2                             0x00001608   Number         4  l298n.o(.text.Motor_UpdatePWM_B)
    [Anonymous Symbol]                       0x0000160c   Section        0  no_mcu_ganv_grayscale_sensor.o(.text.No_MCU_Ganv_Sensor_Init)
    __arm_cp.6_0                             0x00001790   Number         4  no_mcu_ganv_grayscale_sensor.o(.text.No_MCU_Ganv_Sensor_Init)
    [Anonymous Symbol]                       0x00001794   Section        0  no_mcu_ganv_grayscale_sensor.o(.text.No_MCU_Ganv_Sensor_Init_Frist)
    [Anonymous Symbol]                       0x00001806   Section        0  no_mcu_ganv_grayscale_sensor.o(.text.No_Mcu_Ganv_Sensor_Task_Without_tick)
    [Anonymous Symbol]                       0x00001848   Section        0  pid.o(.text.Pid_Yaw)
    __arm_cp.0_0                             0x00001920   Number         4  pid.o(.text.Pid_Yaw)
    __arm_cp.0_1                             0x00001924   Number         4  pid.o(.text.Pid_Yaw)
    __arm_cp.0_2                             0x00001928   Number         4  pid.o(.text.Pid_Yaw)
    __arm_cp.0_3                             0x0000192c   Number         4  pid.o(.text.Pid_Yaw)
    __arm_cp.0_4                             0x00001930   Number         4  pid.o(.text.Pid_Yaw)
    __arm_cp.0_5                             0x00001934   Number         4  pid.o(.text.Pid_Yaw)
    __arm_cp.0_6                             0x00001938   Number         4  pid.o(.text.Pid_Yaw)
    __arm_cp.0_7                             0x0000193c   Number         4  pid.o(.text.Pid_Yaw)
    __arm_cp.0_8                             0x00001940   Number         4  pid.o(.text.Pid_Yaw)
    __arm_cp.0_9                             0x00001944   Number         4  pid.o(.text.Pid_Yaw)
    [Anonymous Symbol]                       0x00001948   Section        0  ti_msp_dl_config.o(.text.SYSCFG_DL_ADC_VOLTAGE_init)
    __arm_cp.6_0                             0x000019ac   Number         4  ti_msp_dl_config.o(.text.SYSCFG_DL_ADC_VOLTAGE_init)
    [Anonymous Symbol]                       0x000019b0   Section        0  ti_msp_dl_config.o(.text.SYSCFG_DL_DMA_CH0_init)
    __arm_cp.42_0                            0x000019d0   Number         4  ti_msp_dl_config.o(.text.SYSCFG_DL_DMA_CH0_init)
    __arm_cp.42_1                            0x000019d4   Number         4  ti_msp_dl_config.o(.text.SYSCFG_DL_DMA_CH0_init)
    [Anonymous Symbol]                       0x000019d8   Section        0  ti_msp_dl_config.o(.text.SYSCFG_DL_DMA_init)
    [Anonymous Symbol]                       0x000019e0   Section        0  ti_msp_dl_config.o(.text.SYSCFG_DL_GPIO_init)
    __arm_cp.2_1                             0x00001a84   Number         4  ti_msp_dl_config.o(.text.SYSCFG_DL_GPIO_init)
    [Anonymous Symbol]                       0x00001a88   Section        0  ti_msp_dl_config.o(.text.SYSCFG_DL_SYSCTL_init)
    [Anonymous Symbol]                       0x00001aaa   Section        0  ti_msp_dl_config.o(.text.SYSCFG_DL_SYSTICK_init)
    [Anonymous Symbol]                       0x00001ab8   Section        0  ti_msp_dl_config.o(.text.SYSCFG_DL_TIMER_0_init)
    __arm_cp.4_0                             0x00001ae8   Number         4  ti_msp_dl_config.o(.text.SYSCFG_DL_TIMER_0_init)
    __arm_cp.4_2                             0x00001aec   Number         4  ti_msp_dl_config.o(.text.SYSCFG_DL_TIMER_0_init)
    [Anonymous Symbol]                       0x00001af0   Section        0  ti_msp_dl_config.o(.text.SYSCFG_DL_UART_0_init)
    __arm_cp.5_0                             0x00001b24   Number         4  ti_msp_dl_config.o(.text.SYSCFG_DL_UART_0_init)
    __arm_cp.5_2                             0x00001b28   Number         4  ti_msp_dl_config.o(.text.SYSCFG_DL_UART_0_init)
    [Anonymous Symbol]                       0x00001b2c   Section        0  ti_msp_dl_config.o(.text.SYSCFG_DL_init)
    [Anonymous Symbol]                       0x00001b50   Section        0  ti_msp_dl_config.o(.text.SYSCFG_DL_initPower)
    __arm_cp.1_0                             0x00001b98   Number         4  ti_msp_dl_config.o(.text.SYSCFG_DL_initPower)
    __arm_cp.1_1                             0x00001b9c   Number         4  ti_msp_dl_config.o(.text.SYSCFG_DL_initPower)
    __arm_cp.1_3                             0x00001ba0   Number         4  ti_msp_dl_config.o(.text.SYSCFG_DL_initPower)
    SysTick_Config                           0x00001ba5   Thumb Code    68  ti_msp_dl_config.o(.text.SysTick_Config)
    [Anonymous Symbol]                       0x00001ba4   Section        0  ti_msp_dl_config.o(.text.SysTick_Config)
    __arm_cp.44_0                            0x00001be8   Number         4  ti_msp_dl_config.o(.text.SysTick_Config)
    __arm_cp.44_1                            0x00001bec   Number         4  ti_msp_dl_config.o(.text.SysTick_Config)
    __arm_cp.44_2                            0x00001bf0   Number         4  ti_msp_dl_config.o(.text.SysTick_Config)
    [Anonymous Symbol]                       0x00001bf4   Section        0  delay.o(.text.SysTick_Handler)
    [Anonymous Symbol]                       0x00001bfc   Section        0  l298n.o(.text.TIMG0_IRQHandler)
    [Anonymous Symbol]                       0x00001c08   Section        0  delay.o(.text.Tick_SysTickCallback)
    [Anonymous Symbol]                       0x00001c14   Section        0  delay.o(.text.Tick_delay)
    __arm_cp.3_0                             0x00001c38   Number         4  delay.o(.text.Tick_delay)
    __NVIC_EnableIRQ                         0x00001c3d   Thumb Code    40  main.o(.text.__NVIC_EnableIRQ)
    [Anonymous Symbol]                       0x00001c3c   Section        0  main.o(.text.__NVIC_EnableIRQ)
    __arm_cp.9_0                             0x00001c64   Number         4  main.o(.text.__NVIC_EnableIRQ)
    __NVIC_SetPriority                       0x00001c69   Thumb Code   124  ti_msp_dl_config.o(.text.__NVIC_SetPriority)
    [Anonymous Symbol]                       0x00001c68   Section        0  ti_msp_dl_config.o(.text.__NVIC_SetPriority)
    __arm_cp.29_0                            0x00001ce4   Number         4  ti_msp_dl_config.o(.text.__NVIC_SetPriority)
    __arm_cp.29_1                            0x00001ce8   Number         4  ti_msp_dl_config.o(.text.__NVIC_SetPriority)
    [Anonymous Symbol]                       0x00001cec   Section        0  adc.o(.text.adc_getValue)
    [Anonymous Symbol]                       0x00001d5c   Section        0  no_mcu_ganv_grayscale_sensor.o(.text.convertAnalogToDigital)
    [Anonymous Symbol]                       0x00001dc8   Section        0  delay.o(.text.delay_us)
    [Anonymous Symbol]                       0x00001de8   Section        0  main.o(.text.fputc)
    __arm_cp.0_0                             0x00001e10   Number         4  main.o(.text.fputc)
    [Anonymous Symbol]                       0x00001e14   Section        0  main.o(.text.main)
    __arm_cp.4_0                             0x00001eb0   Number         4  main.o(.text.main)
    __arm_cp.4_1                             0x00001eb4   Number         4  main.o(.text.main)
    __arm_cp.4_2                             0x00001eb8   Number         4  main.o(.text.main)
    __arm_cp.4_3                             0x00001ebc   Number         4  main.o(.text.main)
    __arm_cp.4_4                             0x00001ec0   Number         4  main.o(.text.main)
    __arm_cp.4_5                             0x00001ec4   Number         4  main.o(.text.main)
    __arm_cp.4_6                             0x00001ec8   Number         4  main.o(.text.main)
    __arm_cp.4_7                             0x00001ecc   Number         4  main.o(.text.main)
    __arm_cp.4_8                             0x00001ed0   Number         4  main.o(.text.main)
    __arm_cp.4_9                             0x00001ed4   Number         4  main.o(.text.main)
    __arm_cp.4_10                            0x00001ed8   Number         4  main.o(.text.main)
    __arm_cp.4_11                            0x00001edc   Number         4  main.o(.text.main)
    __arm_cp.4_12                            0x00001ee0   Number         4  main.o(.text.main)
    [Anonymous Symbol]                       0x00001ee4   Section        0  no_mcu_ganv_grayscale_sensor.o(.text.normalizeAnalogValues)
    i.__0printf                              0x00001f90   Section        0  printfa.o(i.__0printf)
    i.__ARM_clz                              0x00001fb0   Section        0  depilogue.o(i.__ARM_clz)
    i.__scatterload_copy                     0x00001fe0   Section       14  handlers.o(i.__scatterload_copy)
    i.__scatterload_null                     0x00001ff0   Section        2  handlers.o(i.__scatterload_null)
    i.__scatterload_zeroinit                 0x00001ff8   Section       14  handlers.o(i.__scatterload_zeroinit)
    _fp_digits                               0x00002009   Thumb Code   344  printfa.o(i._fp_digits)
    i._fp_digits                             0x00002008   Section        0  printfa.o(i._fp_digits)
    _printf_core                             0x0000217d   Thumb Code  1754  printfa.o(i._printf_core)
    i._printf_core                           0x0000217c   Section        0  printfa.o(i._printf_core)
    _printf_post_padding                     0x00002869   Thumb Code    32  printfa.o(i._printf_post_padding)
    i._printf_post_padding                   0x00002868   Section        0  printfa.o(i._printf_post_padding)
    _printf_pre_padding                      0x00002889   Thumb Code    44  printfa.o(i._printf_pre_padding)
    i._printf_pre_padding                    0x00002888   Section        0  printfa.o(i._printf_pre_padding)
    gADC_VOLTAGEClockConfig                  0x000028b4   Data           8  ti_msp_dl_config.o(.rodata.gADC_VOLTAGEClockConfig)
    [Anonymous Symbol]                       0x000028b4   Section        0  ti_msp_dl_config.o(.rodata.gADC_VOLTAGEClockConfig)
    gDMA_CH0Config                           0x000028bc   Data          24  ti_msp_dl_config.o(.rodata.gDMA_CH0Config)
    [Anonymous Symbol]                       0x000028bc   Section        0  ti_msp_dl_config.o(.rodata.gDMA_CH0Config)
    gTIMER_0ClockConfig                      0x000028d4   Data           3  ti_msp_dl_config.o(.rodata.gTIMER_0ClockConfig)
    [Anonymous Symbol]                       0x000028d4   Section        0  ti_msp_dl_config.o(.rodata.gTIMER_0ClockConfig)
    gTIMER_0TimerConfig                      0x000028d8   Data          20  ti_msp_dl_config.o(.rodata.gTIMER_0TimerConfig)
    [Anonymous Symbol]                       0x000028d8   Section        0  ti_msp_dl_config.o(.rodata.gTIMER_0TimerConfig)
    gUART_0ClockConfig                       0x000028ec   Data           2  ti_msp_dl_config.o(.rodata.gUART_0ClockConfig)
    [Anonymous Symbol]                       0x000028ec   Section        0  ti_msp_dl_config.o(.rodata.gUART_0ClockConfig)
    gUART_0Config                            0x000028ee   Data          10  ti_msp_dl_config.o(.rodata.gUART_0Config)
    [Anonymous Symbol]                       0x000028ee   Section        0  ti_msp_dl_config.o(.rodata.gUART_0Config)
    [Anonymous Symbol]                       0x000028f8   Section        0  main.o(.rodata.str1.1)
    .data                                    0x20000000   Section        4  stdout.o(.data)
    CalculateNormalizedValue.last_value      0x20000088   Data           4  main.o(.bss.CalculateNormalizedValue.last_value)
    [Anonymous Symbol]                       0x20000088   Section        0  main.o(.bss.CalculateNormalizedValue.last_value)
    STACK                                    0x20000198   Section     3328  startup_mspm0l130x_uvision.o(STACK)

    Global Symbols

    Symbol Name                              Value     Ov Type        Size  Object(Section)

    BuildAttributes$$THM_ISAv3M$S$PE$A:L22$X:L11$S22$IEEE1$IW$~IW$USESV6$~STKCKD$USESV7$~SHL$OTIME$ROPI$EBA8$MICROLIB$REQ8$PRES8$EABIv2 0x00000000   Number         0  anon$$obj.o ABSOLUTE
    __Vectors                                0x00000000   Data           4  startup_mspm0l130x_uvision.o(RESET)
    __cpp_initialize__aeabi_                  - Undefined Weak Reference
    __cxa_finalize                            - Undefined Weak Reference
    __decompress                              - Undefined Weak Reference
    _clock_init                               - Undefined Weak Reference
    _microlib_exit                            - Undefined Weak Reference
    __Vectors_End                            0x000000c0   Data           0  startup_mspm0l130x_uvision.o(RESET)
    __Vectors_Size                           0x000000c0   Number         0  startup_mspm0l130x_uvision.o ABSOLUTE
    __main                                   0x000000c1   Thumb Code     0  entry.o(.ARM.Collect$$$$00000000)
    _main_stk                                0x000000c1   Thumb Code     0  entry2.o(.ARM.Collect$$$$00000001)
    _main_scatterload                        0x000000c5   Thumb Code     0  entry5.o(.ARM.Collect$$$$00000004)
    __main_after_scatterload                 0x000000c9   Thumb Code     0  entry5.o(.ARM.Collect$$$$00000004)
    _main_clock                              0x000000c9   Thumb Code     0  entry7b.o(.ARM.Collect$$$$00000008)
    _main_cpp_init                           0x000000c9   Thumb Code     0  entry8b.o(.ARM.Collect$$$$0000000A)
    _main_init                               0x000000c9   Thumb Code     0  entry9a.o(.ARM.Collect$$$$0000000B)
    __rt_final_cpp                           0x000000d1   Thumb Code     0  entry10a.o(.ARM.Collect$$$$0000000D)
    __rt_final_exit                          0x000000d1   Thumb Code     0  entry11a.o(.ARM.Collect$$$$0000000F)
    Reset_Handler                            0x000000d5   Thumb Code     4  startup_mspm0l130x_uvision.o(.text)
    NMI_Handler                              0x000000d9   Thumb Code     2  startup_mspm0l130x_uvision.o(.text)
    HardFault_Handler                        0x000000db   Thumb Code     2  startup_mspm0l130x_uvision.o(.text)
    SVC_Handler                              0x000000dd   Thumb Code     2  startup_mspm0l130x_uvision.o(.text)
    PendSV_Handler                           0x000000df   Thumb Code     2  startup_mspm0l130x_uvision.o(.text)
    ADC0_IRQHandler                          0x000000e3   Thumb Code     0  startup_mspm0l130x_uvision.o(.text)
    DMA_IRQHandler                           0x000000e3   Thumb Code     0  startup_mspm0l130x_uvision.o(.text)
    Default_Handler                          0x000000e3   Thumb Code     2  startup_mspm0l130x_uvision.o(.text)
    GROUP0_IRQHandler                        0x000000e3   Thumb Code     0  startup_mspm0l130x_uvision.o(.text)
    I2C0_IRQHandler                          0x000000e3   Thumb Code     0  startup_mspm0l130x_uvision.o(.text)
    I2C1_IRQHandler                          0x000000e3   Thumb Code     0  startup_mspm0l130x_uvision.o(.text)
    SPI0_IRQHandler                          0x000000e3   Thumb Code     0  startup_mspm0l130x_uvision.o(.text)
    TIMG1_IRQHandler                         0x000000e3   Thumb Code     0  startup_mspm0l130x_uvision.o(.text)
    TIMG2_IRQHandler                         0x000000e3   Thumb Code     0  startup_mspm0l130x_uvision.o(.text)
    TIMG4_IRQHandler                         0x000000e3   Thumb Code     0  startup_mspm0l130x_uvision.o(.text)
    UART0_IRQHandler                         0x000000e3   Thumb Code     0  startup_mspm0l130x_uvision.o(.text)
    UART1_IRQHandler                         0x000000e3   Thumb Code     0  startup_mspm0l130x_uvision.o(.text)
    __aeabi_memcpy                           0x000000e9   Thumb Code    36  memcpya.o(.text)
    __aeabi_memcpy4                          0x000000e9   Thumb Code     0  memcpya.o(.text)
    __aeabi_memcpy8                          0x000000e9   Thumb Code     0  memcpya.o(.text)
    __aeabi_memset                           0x0000010d   Thumb Code    14  memseta.o(.text)
    __aeabi_memset4                          0x0000010d   Thumb Code     0  memseta.o(.text)
    __aeabi_memset8                          0x0000010d   Thumb Code     0  memseta.o(.text)
    __aeabi_memclr                           0x0000011b   Thumb Code     4  memseta.o(.text)
    __aeabi_memclr4                          0x0000011b   Thumb Code     0  memseta.o(.text)
    __aeabi_memclr8                          0x0000011b   Thumb Code     0  memseta.o(.text)
    _memset$wrapper                          0x0000011f   Thumb Code    18  memseta.o(.text)
    __aeabi_fadd                             0x00000131   Thumb Code   162  fadd.o(.text)
    __aeabi_fsub                             0x000001d3   Thumb Code     8  fadd.o(.text)
    __aeabi_frsub                            0x000001db   Thumb Code     8  fadd.o(.text)
    __aeabi_dadd                             0x000001e5   Thumb Code   328  dadd.o(.text)
    __aeabi_dsub                             0x0000032d   Thumb Code    12  dadd.o(.text)
    __aeabi_drsub                            0x00000339   Thumb Code    12  dadd.o(.text)
    __aeabi_dmul                             0x00000349   Thumb Code   202  dmul.o(.text)
    __aeabi_ddiv                             0x00000419   Thumb Code   234  ddiv.o(.text)
    __aeabi_dcmple                           0x00000509   Thumb Code    44  dcmple.o(.text)
    __aeabi_i2f                              0x00000535   Thumb Code    22  fflti.o(.text)
    __aeabi_i2d                              0x0000054d   Thumb Code    34  dflti.o(.text)
    __aeabi_ui2d                             0x00000575   Thumb Code    24  dfltui.o(.text)
    __aeabi_f2iz                             0x00000591   Thumb Code    50  ffixi.o(.text)
    __aeabi_d2iz                             0x000005c5   Thumb Code    62  dfixi.o(.text)
    __aeabi_uidiv                            0x0000060d   Thumb Code     0  uidiv_div0.o(.text)
    __aeabi_uidivmod                         0x0000060d   Thumb Code    62  uidiv_div0.o(.text)
    __aeabi_idiv                             0x0000064d   Thumb Code     0  idiv_div0.o(.text)
    __aeabi_idivmod                          0x0000064d   Thumb Code    74  idiv_div0.o(.text)
    __aeabi_uldivmod                         0x0000069d   Thumb Code    96  uldiv.o(.text)
    __aeabi_llsl                             0x000006fd   Thumb Code    32  llshl.o(.text)
    _ll_shift_l                              0x000006fd   Thumb Code     0  llshl.o(.text)
    __aeabi_llsr                             0x0000071d   Thumb Code    34  llushr.o(.text)
    _ll_ushift_r                             0x0000071d   Thumb Code     0  llushr.o(.text)
    __aeabi_lasr                             0x0000073f   Thumb Code    38  llsshr.o(.text)
    _ll_sshift_r                             0x0000073f   Thumb Code     0  llsshr.o(.text)
    __I$use$fp                               0x00000765   Thumb Code     0  iusefp.o(.text)
    _float_round                             0x00000765   Thumb Code    16  fepilogue.o(.text)
    _float_epilogue                          0x00000775   Thumb Code   114  fepilogue.o(.text)
    _double_round                            0x000007e7   Thumb Code    26  depilogue.o(.text)
    _double_epilogue                         0x00000801   Thumb Code   164  depilogue.o(.text)
    __aeabi_d2ulz                            0x000008a5   Thumb Code    54  dfixul.o(.text)
    __aeabi_cdrcmple                         0x000008e5   Thumb Code    38  cdrcmple.o(.text)
    __scatterload                            0x00000911   Thumb Code    38  init.o(.text)
    __scatterload_rt2                        0x00000911   Thumb Code     0  init.o(.text)
    CalculateNormalizedValue                 0x00000941   Thumb Code   208  main.o(.text.CalculateNormalizedValue)
    DL_ADC12_setClockConfig                  0x00000b1d   Thumb Code    64  dl_adc12.o(.text.DL_ADC12_setClockConfig)
    DL_Common_delayCycles                    0x00000bbd   Thumb Code    10  dl_common.o(.text.DL_Common_delayCycles)
    DL_DMA_initChannel                       0x00000c15   Thumb Code    68  dl_dma.o(.text.DL_DMA_initChannel)
    DL_Timer_initTimerMode                   0x00000f05   Thumb Code   236  dl_timer.o(.text.DL_Timer_initTimerMode)
    DL_Timer_setClockConfig                  0x00001001   Thumb Code    28  dl_timer.o(.text.DL_Timer_setClockConfig)
    DL_UART_init                             0x00001065   Thumb Code    72  dl_uart.o(.text.DL_UART_init)
    DL_UART_setClockConfig                   0x00001129   Thumb Code    18  dl_uart.o(.text.DL_UART_setClockConfig)
    GROUP1_IRQHandler                        0x00001171   Thumb Code    92  key.o(.text.GROUP1_IRQHandler)
    Get_Analog_value                         0x000011dd   Thumb Code   184  no_mcu_ganv_grayscale_sensor.o(.text.Get_Analog_value)
    Get_Digtal_For_User                      0x00001295   Thumb Code    14  no_mcu_ganv_grayscale_sensor.o(.text.Get_Digtal_For_User)
    Get_Normalize_For_User                   0x000012a3   Thumb Code    56  no_mcu_ganv_grayscale_sensor.o(.text.Get_Normalize_For_User)
    Motor_Control                            0x000012dd   Thumb Code   296  l298n.o(.text.Motor_Control)
    Motor_SetDuty_A                          0x0000142d   Thumb Code    56  l298n.o(.text.Motor_SetDuty_A)
    Motor_SetDuty_B                          0x00001465   Thumb Code    56  l298n.o(.text.Motor_SetDuty_B)
    Motor_UpdatePWM_A                        0x0000149d   Thumb Code   160  l298n.o(.text.Motor_UpdatePWM_A)
    Motor_UpdatePWM_B                        0x00001549   Thumb Code   184  l298n.o(.text.Motor_UpdatePWM_B)
    No_MCU_Ganv_Sensor_Init                  0x0000160d   Thumb Code   388  no_mcu_ganv_grayscale_sensor.o(.text.No_MCU_Ganv_Sensor_Init)
    No_MCU_Ganv_Sensor_Init_Frist            0x00001795   Thumb Code   114  no_mcu_ganv_grayscale_sensor.o(.text.No_MCU_Ganv_Sensor_Init_Frist)
    No_Mcu_Ganv_Sensor_Task_Without_tick     0x00001807   Thumb Code    66  no_mcu_ganv_grayscale_sensor.o(.text.No_Mcu_Ganv_Sensor_Task_Without_tick)
    Pid_Yaw                                  0x00001849   Thumb Code   216  pid.o(.text.Pid_Yaw)
    SYSCFG_DL_ADC_VOLTAGE_init               0x00001949   Thumb Code   100  ti_msp_dl_config.o(.text.SYSCFG_DL_ADC_VOLTAGE_init)
    SYSCFG_DL_DMA_CH0_init                   0x000019b1   Thumb Code    32  ti_msp_dl_config.o(.text.SYSCFG_DL_DMA_CH0_init)
    SYSCFG_DL_DMA_init                       0x000019d9   Thumb Code     8  ti_msp_dl_config.o(.text.SYSCFG_DL_DMA_init)
    SYSCFG_DL_GPIO_init                      0x000019e1   Thumb Code   164  ti_msp_dl_config.o(.text.SYSCFG_DL_GPIO_init)
    SYSCFG_DL_SYSCTL_init                    0x00001a89   Thumb Code    34  ti_msp_dl_config.o(.text.SYSCFG_DL_SYSCTL_init)
    SYSCFG_DL_SYSTICK_init                   0x00001aab   Thumb Code    12  ti_msp_dl_config.o(.text.SYSCFG_DL_SYSTICK_init)
    SYSCFG_DL_TIMER_0_init                   0x00001ab9   Thumb Code    48  ti_msp_dl_config.o(.text.SYSCFG_DL_TIMER_0_init)
    SYSCFG_DL_UART_0_init                    0x00001af1   Thumb Code    52  ti_msp_dl_config.o(.text.SYSCFG_DL_UART_0_init)
    SYSCFG_DL_init                           0x00001b2d   Thumb Code    36  ti_msp_dl_config.o(.text.SYSCFG_DL_init)
    SYSCFG_DL_initPower                      0x00001b51   Thumb Code    72  ti_msp_dl_config.o(.text.SYSCFG_DL_initPower)
    SysTick_Handler                          0x00001bf5   Thumb Code     8  delay.o(.text.SysTick_Handler)
    TIMG0_IRQHandler                         0x00001bfd   Thumb Code    12  l298n.o(.text.TIMG0_IRQHandler)
    Tick_SysTickCallback                     0x00001c09   Thumb Code    12  delay.o(.text.Tick_SysTickCallback)
    Tick_delay                               0x00001c15   Thumb Code    36  delay.o(.text.Tick_delay)
    adc_getValue                             0x00001ced   Thumb Code   112  adc.o(.text.adc_getValue)
    convertAnalogToDigital                   0x00001d5d   Thumb Code   108  no_mcu_ganv_grayscale_sensor.o(.text.convertAnalogToDigital)
    delay_us                                 0x00001dc9   Thumb Code    30  delay.o(.text.delay_us)
    fputc                                    0x00001de9   Thumb Code    40  main.o(.text.fputc)
    main                                     0x00001e15   Thumb Code   156  main.o(.text.main)
    normalizeAnalogValues                    0x00001ee5   Thumb Code   170  no_mcu_ganv_grayscale_sensor.o(.text.normalizeAnalogValues)
    __0printf                                0x00001f91   Thumb Code    24  printfa.o(i.__0printf)
    __1printf                                0x00001f91   Thumb Code     0  printfa.o(i.__0printf)
    __2printf                                0x00001f91   Thumb Code     0  printfa.o(i.__0printf)
    __c89printf                              0x00001f91   Thumb Code     0  printfa.o(i.__0printf)
    printf                                   0x00001f91   Thumb Code     0  printfa.o(i.__0printf)
    __ARM_clz                                0x00001fb1   Thumb Code    46  depilogue.o(i.__ARM_clz)
    __scatterload_copy                       0x00001fe1   Thumb Code    14  handlers.o(i.__scatterload_copy)
    __scatterload_null                       0x00001ff1   Thumb Code     2  handlers.o(i.__scatterload_null)
    __scatterload_zeroinit                   0x00001ff9   Thumb Code    14  handlers.o(i.__scatterload_zeroinit)
    Region$$Table$$Base                      0x00002900   Number         0  anon$$obj.o(Region$$Table)
    Region$$Table$$Limit                     0x00002920   Number         0  anon$$obj.o(Region$$Table)
    __stdout                                 0x20000000   Data           4  stdout.o(.data)
    K_V                                      0x20000004   Data           4  l298n.o(.data.K_V)
    Kd_Yaw                                   0x20000008   Data           4  pid.o(.data.Kd_Yaw)
    Kp_Yaw                                   0x2000000c   Data           4  pid.o(.data.Kp_Yaw)
    black                                    0x20000010   Data          16  main.o(.data.black)
    max                                      0x20000020   Data           4  pid.o(.data.max)
    motorDuty_A                              0x20000024   Data           2  l298n.o(.data.motorDuty_A)
    motorDuty_B                              0x20000026   Data           2  l298n.o(.data.motorDuty_B)
    white                                    0x20000028   Data          16  main.o(.data.white)
    ADC_VALUE                                0x20000038   Data          80  adc.o(.bss.ADC_VALUE)
    Digtal                                   0x2000008c   Data           1  main.o(.bss.Digtal)
    Err_Yaw                                  0x20000090   Data           4  pid.o(.bss.Err_Yaw)
    Integral_Yaw                             0x20000094   Data           4  pid.o(.bss.Integral_Yaw)
    Ki_Yaw                                   0x20000098   Data           4  pid.o(.bss.Ki_Yaw)
    LastErr_Yaw                              0x2000009c   Data           4  pid.o(.bss.LastErr_Yaw)
    Normal                                   0x200000a0   Data          16  main.o(.bss.Normal)
    Output_Yaw                               0x200000b0   Data           4  pid.o(.bss.Output_Yaw)
    SpeedL                                   0x200000b4   Data           4  l298n.o(.bss.SpeedL)
    SpeedR                                   0x200000b8   Data           4  l298n.o(.bss.SpeedR)
    Speed_Set                                0x200000bc   Data           4  l298n.o(.bss.Speed_Set)
    Tarangle                                 0x200000c0   Data           4  l298n.o(.bss.Tarangle)
    Tick                                     0x200000c4   Data           4  delay.o(.bss.Tick)
    Yaw_Now_Correct                          0x200000c8   Data           4  pid.o(.bss.Yaw_Now_Correct)
    key_pressed                              0x200000cc   Data           1  key.o(.bss.key_pressed)
    key_start_pressed                        0x200000cd   Data           1  key.o(.bss.key_start_pressed)
    last_key_time                            0x200000d0   Data           4  key.o(.bss.last_key_time)
    pwmCounter_A                             0x200000d4   Data           1  l298n.o(.bss.pwmCounter_A)
    pwmCounter_B                             0x200000d5   Data           1  l298n.o(.bss.pwmCounter_B)
    pwmL                                     0x200000d8   Data           4  l298n.o(.bss.pwmL)
    pwmR                                     0x200000dc   Data           4  l298n.o(.bss.pwmR)
    result_angle                             0x200000e0   Data           4  pid.o(.bss.result_angle)
    sensor                                   0x200000e8   Data         176  main.o(.bss.sensor)
    __initial_sp                             0x20000e98   Data           0  startup_mspm0l130x_uvision.o(STACK)



==============================================================================

Memory Map of the image

  Image Entry point : 0x000000c1

  Load Region LR_IROM1 (Base: 0x00000000, Size: 0x00002958, Max: 0x0000fff8, ABSOLUTE)

    Execution Region ER_IROM1 (Exec base: 0x00000000, Load base: 0x00000000, Size: 0x00002920, Max: 0x0000fff8, ABSOLUTE)

    Exec Addr    Load Addr    Size         Type   Attr      Idx    E Section Name        Object

    0x00000000   0x00000000   0x000000c0   Data   RO           42    RESET               startup_mspm0l130x_uvision.o
    0x000000c0   0x000000c0   0x00000000   Code   RO          450  * .ARM.Collect$$$$00000000  mc_p.l(entry.o)
    0x000000c0   0x000000c0   0x00000004   Code   RO          522    .ARM.Collect$$$$00000001  mc_p.l(entry2.o)
    0x000000c4   0x000000c4   0x00000004   Code   RO          525    .ARM.Collect$$$$00000004  mc_p.l(entry5.o)
    0x000000c8   0x000000c8   0x00000000   Code   RO          527    .ARM.Collect$$$$00000008  mc_p.l(entry7b.o)
    0x000000c8   0x000000c8   0x00000000   Code   RO          529    .ARM.Collect$$$$0000000A  mc_p.l(entry8b.o)
    0x000000c8   0x000000c8   0x00000008   Code   RO          530    .ARM.Collect$$$$0000000B  mc_p.l(entry9a.o)
    0x000000d0   0x000000d0   0x00000000   Code   RO          532    .ARM.Collect$$$$0000000D  mc_p.l(entry10a.o)
    0x000000d0   0x000000d0   0x00000000   Code   RO          534    .ARM.Collect$$$$0000000F  mc_p.l(entry11a.o)
    0x000000d0   0x000000d0   0x00000004   Code   RO          523    .ARM.Collect$$$$00002712  mc_p.l(entry2.o)
    0x000000d4   0x000000d4   0x00000014   Code   RO           43    .text               startup_mspm0l130x_uvision.o
    0x000000e8   0x000000e8   0x00000024   Code   RO          468    .text               mc_p.l(memcpya.o)
    0x0000010c   0x0000010c   0x00000024   Code   RO          470    .text               mc_p.l(memseta.o)
    0x00000130   0x00000130   0x000000b2   Code   RO          502    .text               mf_p.l(fadd.o)
    0x000001e2   0x000001e2   0x00000002   PAD
    0x000001e4   0x000001e4   0x00000164   Code   RO          504    .text               mf_p.l(dadd.o)
    0x00000348   0x00000348   0x000000d0   Code   RO          506    .text               mf_p.l(dmul.o)
    0x00000418   0x00000418   0x000000f0   Code   RO          508    .text               mf_p.l(ddiv.o)
    0x00000508   0x00000508   0x0000002c   Code   RO          510    .text               mf_p.l(dcmple.o)
    0x00000534   0x00000534   0x00000016   Code   RO          512    .text               mf_p.l(fflti.o)
    0x0000054a   0x0000054a   0x00000002   PAD
    0x0000054c   0x0000054c   0x00000028   Code   RO          514    .text               mf_p.l(dflti.o)
    0x00000574   0x00000574   0x0000001c   Code   RO          516    .text               mf_p.l(dfltui.o)
    0x00000590   0x00000590   0x00000032   Code   RO          518    .text               mf_p.l(ffixi.o)
    0x000005c2   0x000005c2   0x00000002   PAD
    0x000005c4   0x000005c4   0x00000048   Code   RO          520    .text               mf_p.l(dfixi.o)
    0x0000060c   0x0000060c   0x0000003e   Code   RO          540    .text               mc_p.l(uidiv_div0.o)
    0x0000064a   0x0000064a   0x00000002   PAD
    0x0000064c   0x0000064c   0x00000050   Code   RO          542    .text               mc_p.l(idiv_div0.o)
    0x0000069c   0x0000069c   0x00000060   Code   RO          546    .text               mc_p.l(uldiv.o)
    0x000006fc   0x000006fc   0x00000020   Code   RO          548    .text               mc_p.l(llshl.o)
    0x0000071c   0x0000071c   0x00000022   Code   RO          550    .text               mc_p.l(llushr.o)
    0x0000073e   0x0000073e   0x00000026   Code   RO          552    .text               mc_p.l(llsshr.o)
    0x00000764   0x00000764   0x00000000   Code   RO          554    .text               mc_p.l(iusefp.o)
    0x00000764   0x00000764   0x00000082   Code   RO          555    .text               mf_p.l(fepilogue.o)
    0x000007e6   0x000007e6   0x000000be   Code   RO          557    .text               mf_p.l(depilogue.o)
    0x000008a4   0x000008a4   0x00000040   Code   RO          561    .text               mf_p.l(dfixul.o)
    0x000008e4   0x000008e4   0x00000028   Code   RO          563    .text               mf_p.l(cdrcmple.o)
    0x0000090c   0x0000090c   0x00000004   PAD
    0x00000910   0x00000910   0x00000030   Code   RO          565    .text               mc_p.l(init.o)
    0x00000940   0x00000940   0x000000e0   Code   RO            8    .text.CalculateNormalizedValue  main.o
    0x00000a20   0x00000a20   0x0000004a   Code   RO          122    .text.DL_ADC12_configConversionMem  ti_msp_dl_config.o
    0x00000a6a   0x00000a6a   0x00000016   Code   RO          132    .text.DL_ADC12_enableConversions  ti_msp_dl_config.o
    0x00000a80   0x00000a80   0x00000018   Code   RO          126    .text.DL_ADC12_enableDMA  ti_msp_dl_config.o
    0x00000a98   0x00000a98   0x0000001c   Code   RO          130    .text.DL_ADC12_enableDMATrigger  ti_msp_dl_config.o
    0x00000ab4   0x00000ab4   0x00000014   Code   RO           82    .text.DL_ADC12_enablePower  ti_msp_dl_config.o
    0x00000ac8   0x00000ac8   0x00000044   Code   RO          120    .text.DL_ADC12_initSingleSample  ti_msp_dl_config.o
    0x00000b0c   0x00000b0c   0x00000010   Code   RO           74    .text.DL_ADC12_reset  ti_msp_dl_config.o
    0x00000b1c   0x00000b1c   0x00000040   Code   RO          307    .text.DL_ADC12_setClockConfig  driverlib.a(dl_adc12.o)
    0x00000b5c   0x00000b5c   0x0000002c   Code   RO          128    .text.DL_ADC12_setDMASamplesCnt  ti_msp_dl_config.o
    0x00000b88   0x00000b88   0x00000018   Code   RO          124    .text.DL_ADC12_setSampleTime0  ti_msp_dl_config.o
    0x00000ba0   0x00000ba0   0x0000001c   Code   RO           18    .text.DL_ADC12_startConversion  main.o
    0x00000bbc   0x00000bbc   0x0000000a   Code   RO          319    .text.DL_Common_delayCycles  driverlib.a(dl_common.o)
    0x00000bc6   0x00000bc6   0x00000028   Code   RO          140    .text.DL_Common_updateReg  ti_msp_dl_config.o
    0x00000bee   0x00000bee   0x00000026   Code   RO           16    .text.DL_DMA_enableChannel  main.o
    0x00000c14   0x00000c14   0x00000044   Code   RO          328    .text.DL_DMA_initChannel  driverlib.a(dl_dma.o)
    0x00000c58   0x00000c58   0x00000028   Code   RO           14    .text.DL_DMA_setDestAddr  main.o
    0x00000c80   0x00000c80   0x00000028   Code   RO           12    .text.DL_DMA_setSrcAddr  main.o
    0x00000ca8   0x00000ca8   0x00000030   Code   RO          136    .text.DL_DMA_setTransferSize  ti_msp_dl_config.o
    0x00000cd8   0x00000cd8   0x0000001c   Code   RO           98    .text.DL_GPIO_clearInterruptStatus  ti_msp_dl_config.o
    0x00000cf4   0x00000cf4   0x00000014   Code   RO           92    .text.DL_GPIO_clearPins  ti_msp_dl_config.o
    0x00000d08   0x00000d08   0x00000014   Code   RO          184    .text.DL_GPIO_clearPins  no_mcu_ganv_grayscale_sensor.o
    0x00000d1c   0x00000d1c   0x00000014   Code   RO          253    .text.DL_GPIO_clearPins  l298n.o
    0x00000d30   0x00000d30   0x00000018   Code   RO          100    .text.DL_GPIO_enableInterrupt  ti_msp_dl_config.o
    0x00000d48   0x00000d48   0x00000018   Code   RO           94    .text.DL_GPIO_enableOutput  ti_msp_dl_config.o
    0x00000d60   0x00000d60   0x00000018   Code   RO           76    .text.DL_GPIO_enablePower  ti_msp_dl_config.o
    0x00000d78   0x00000d78   0x00000012   Code   RO          215    .text.DL_GPIO_getPendingInterrupt  key.o
    0x00000d8a   0x00000d8a   0x00000002   PAD
    0x00000d8c   0x00000d8c   0x00000030   Code   RO           90    .text.DL_GPIO_initDigitalInputFeatures  ti_msp_dl_config.o
    0x00000dbc   0x00000dbc   0x00000014   Code   RO           88    .text.DL_GPIO_initDigitalOutput  ti_msp_dl_config.o
    0x00000dd0   0x00000dd0   0x0000001c   Code   RO           86    .text.DL_GPIO_initPeripheralInputFunction  ti_msp_dl_config.o
    0x00000dec   0x00000dec   0x0000001c   Code   RO           84    .text.DL_GPIO_initPeripheralOutputFunction  ti_msp_dl_config.o
    0x00000e08   0x00000e08   0x00000016   Code   RO          217    .text.DL_GPIO_readPins  key.o
    0x00000e1e   0x00000e1e   0x00000002   PAD
    0x00000e20   0x00000e20   0x00000018   Code   RO           68    .text.DL_GPIO_reset  ti_msp_dl_config.o
    0x00000e38   0x00000e38   0x00000014   Code   RO          182    .text.DL_GPIO_setPins  no_mcu_ganv_grayscale_sensor.o
    0x00000e4c   0x00000e4c   0x00000018   Code   RO          255    .text.DL_GPIO_setPins  l298n.o
    0x00000e64   0x00000e64   0x00000018   Code   RO           96    .text.DL_GPIO_setUpperPinsPolarity  ti_msp_dl_config.o
    0x00000e7c   0x00000e7c   0x00000010   Code   RO          106    .text.DL_SYSCTL_enableMFPCLK  ti_msp_dl_config.o
    0x00000e8c   0x00000e8c   0x00000018   Code   RO          102    .text.DL_SYSCTL_setBORThreshold  ti_msp_dl_config.o
    0x00000ea4   0x00000ea4   0x0000001c   Code   RO          104    .text.DL_SYSCTL_setSYSOSCFreq  ti_msp_dl_config.o
    0x00000ec0   0x00000ec0   0x00000014   Code   RO          112    .text.DL_Timer_enableClock  ti_msp_dl_config.o
    0x00000ed4   0x00000ed4   0x0000001c   Code   RO          110    .text.DL_Timer_enableInterrupt  ti_msp_dl_config.o
    0x00000ef0   0x00000ef0   0x00000014   Code   RO           78    .text.DL_Timer_enablePower  ti_msp_dl_config.o
    0x00000f04   0x00000f04   0x000000ec   Code   RO          342    .text.DL_Timer_initTimerMode  driverlib.a(dl_timer.o)
    0x00000ff0   0x00000ff0   0x00000010   Code   RO           70    .text.DL_Timer_reset  ti_msp_dl_config.o
    0x00001000   0x00001000   0x0000001c   Code   RO          338    .text.DL_Timer_setClockConfig  driverlib.a(dl_timer.o)
    0x0000101c   0x0000101c   0x00000018   Code   RO           22    .text.DL_Timer_startCounter  main.o
    0x00001034   0x00001034   0x00000016   Code   RO          118    .text.DL_UART_enable  ti_msp_dl_config.o
    0x0000104a   0x0000104a   0x00000002   PAD
    0x0000104c   0x0000104c   0x00000018   Code   RO           80    .text.DL_UART_enablePower  ti_msp_dl_config.o
    0x00001064   0x00001064   0x00000048   Code   RO          411    .text.DL_UART_init  driverlib.a(dl_uart.o)
    0x000010ac   0x000010ac   0x00000018   Code   RO            4    .text.DL_UART_isBusy  main.o
    0x000010c4   0x000010c4   0x00000018   Code   RO           72    .text.DL_UART_reset  ti_msp_dl_config.o
    0x000010dc   0x000010dc   0x0000004c   Code   RO          116    .text.DL_UART_setBaudRateDivisor  ti_msp_dl_config.o
    0x00001128   0x00001128   0x00000012   Code   RO          413    .text.DL_UART_setClockConfig  driverlib.a(dl_uart.o)
    0x0000113a   0x0000113a   0x0000001e   Code   RO          114    .text.DL_UART_setOversampling  ti_msp_dl_config.o
    0x00001158   0x00001158   0x00000016   Code   RO            6    .text.DL_UART_transmitData  main.o
    0x0000116e   0x0000116e   0x00000002   PAD
    0x00001170   0x00001170   0x0000006c   Code   RO          213    .text.GROUP1_IRQHandler  key.o
    0x000011dc   0x000011dc   0x000000b8   Code   RO          180    .text.Get_Analog_value  no_mcu_ganv_grayscale_sensor.o
    0x00001294   0x00001294   0x0000000e   Code   RO          200    .text.Get_Digtal_For_User  no_mcu_ganv_grayscale_sensor.o
    0x000012a2   0x000012a2   0x00000038   Code   RO          202    .text.Get_Normalize_For_User  no_mcu_ganv_grayscale_sensor.o
    0x000012da   0x000012da   0x00000002   PAD
    0x000012dc   0x000012dc   0x00000150   Code   RO          261    .text.Motor_Control  l298n.o
    0x0000142c   0x0000142c   0x00000038   Code   RO          247    .text.Motor_SetDuty_A  l298n.o
    0x00001464   0x00001464   0x00000038   Code   RO          249    .text.Motor_SetDuty_B  l298n.o
    0x0000149c   0x0000149c   0x000000ac   Code   RO          251    .text.Motor_UpdatePWM_A  l298n.o
    0x00001548   0x00001548   0x000000c4   Code   RO          259    .text.Motor_UpdatePWM_B  l298n.o
    0x0000160c   0x0000160c   0x00000188   Code   RO          192    .text.No_MCU_Ganv_Sensor_Init  no_mcu_ganv_grayscale_sensor.o
    0x00001794   0x00001794   0x00000072   Code   RO          190    .text.No_MCU_Ganv_Sensor_Init_Frist  no_mcu_ganv_grayscale_sensor.o
    0x00001806   0x00001806   0x00000042   Code   RO          194    .text.No_Mcu_Ganv_Sensor_Task_Without_tick  no_mcu_ganv_grayscale_sensor.o
    0x00001848   0x00001848   0x00000100   Code   RO          229    .text.Pid_Yaw       pid.o
    0x00001948   0x00001948   0x00000068   Code   RO           62    .text.SYSCFG_DL_ADC_VOLTAGE_init  ti_msp_dl_config.o
    0x000019b0   0x000019b0   0x00000028   Code   RO          134    .text.SYSCFG_DL_DMA_CH0_init  ti_msp_dl_config.o
    0x000019d8   0x000019d8   0x00000008   Code   RO           64    .text.SYSCFG_DL_DMA_init  ti_msp_dl_config.o
    0x000019e0   0x000019e0   0x000000a8   Code   RO           54    .text.SYSCFG_DL_GPIO_init  ti_msp_dl_config.o
    0x00001a88   0x00001a88   0x00000022   Code   RO           56    .text.SYSCFG_DL_SYSCTL_init  ti_msp_dl_config.o
    0x00001aaa   0x00001aaa   0x0000000c   Code   RO           66    .text.SYSCFG_DL_SYSTICK_init  ti_msp_dl_config.o
    0x00001ab6   0x00001ab6   0x00000002   PAD
    0x00001ab8   0x00001ab8   0x00000038   Code   RO           58    .text.SYSCFG_DL_TIMER_0_init  ti_msp_dl_config.o
    0x00001af0   0x00001af0   0x0000003c   Code   RO           60    .text.SYSCFG_DL_UART_0_init  ti_msp_dl_config.o
    0x00001b2c   0x00001b2c   0x00000024   Code   RO           50    .text.SYSCFG_DL_init  ti_msp_dl_config.o
    0x00001b50   0x00001b50   0x00000054   Code   RO           52    .text.SYSCFG_DL_initPower  ti_msp_dl_config.o
    0x00001ba4   0x00001ba4   0x00000050   Code   RO          138    .text.SysTick_Config  ti_msp_dl_config.o
    0x00001bf4   0x00001bf4   0x00000008   Code   RO          164    .text.SysTick_Handler  delay.o
    0x00001bfc   0x00001bfc   0x0000000c   Code   RO          257    .text.TIMG0_IRQHandler  l298n.o
    0x00001c08   0x00001c08   0x0000000c   Code   RO          166    .text.Tick_SysTickCallback  delay.o
    0x00001c14   0x00001c14   0x00000028   Code   RO          170    .text.Tick_delay    delay.o
    0x00001c3c   0x00001c3c   0x0000002c   Code   RO           20    .text.__NVIC_EnableIRQ  main.o
    0x00001c68   0x00001c68   0x00000084   Code   RO          108    .text.__NVIC_SetPriority  ti_msp_dl_config.o
    0x00001cec   0x00001cec   0x00000070   Code   RO          155    .text.adc_getValue  adc.o
    0x00001d5c   0x00001d5c   0x0000006c   Code   RO          186    .text.convertAnalogToDigital  no_mcu_ganv_grayscale_sensor.o
    0x00001dc8   0x00001dc8   0x0000001e   Code   RO          168    .text.delay_us      delay.o
    0x00001de6   0x00001de6   0x00000002   PAD
    0x00001de8   0x00001de8   0x0000002c   Code   RO            2    .text.fputc         main.o
    0x00001e14   0x00001e14   0x000000d0   Code   RO           10    .text.main          main.o
    0x00001ee4   0x00001ee4   0x000000aa   Code   RO          188    .text.normalizeAnalogValues  no_mcu_ganv_grayscale_sensor.o
    0x00001f8e   0x00001f8e   0x00000002   PAD
    0x00001f90   0x00001f90   0x00000020   Code   RO          475    i.__0printf         mc_p.l(printfa.o)
    0x00001fb0   0x00001fb0   0x0000002e   Code   RO          559    i.__ARM_clz         mf_p.l(depilogue.o)
    0x00001fde   0x00001fde   0x00000002   PAD
    0x00001fe0   0x00001fe0   0x0000000e   Code   RO          569    i.__scatterload_copy  mc_p.l(handlers.o)
    0x00001fee   0x00001fee   0x00000002   PAD
    0x00001ff0   0x00001ff0   0x00000002   Code   RO          570    i.__scatterload_null  mc_p.l(handlers.o)
    0x00001ff2   0x00001ff2   0x00000006   PAD
    0x00001ff8   0x00001ff8   0x0000000e   Code   RO          571    i.__scatterload_zeroinit  mc_p.l(handlers.o)
    0x00002006   0x00002006   0x00000002   PAD
    0x00002008   0x00002008   0x00000174   Code   RO          482    i._fp_digits        mc_p.l(printfa.o)
    0x0000217c   0x0000217c   0x000006ec   Code   RO          483    i._printf_core      mc_p.l(printfa.o)
    0x00002868   0x00002868   0x00000020   Code   RO          484    i._printf_post_padding  mc_p.l(printfa.o)
    0x00002888   0x00002888   0x0000002c   Code   RO          485    i._printf_pre_padding  mc_p.l(printfa.o)
    0x000028b4   0x000028b4   0x00000008   Data   RO          146    .rodata.gADC_VOLTAGEClockConfig  ti_msp_dl_config.o
    0x000028bc   0x000028bc   0x00000018   Data   RO          147    .rodata.gDMA_CH0Config  ti_msp_dl_config.o
    0x000028d4   0x000028d4   0x00000003   Data   RO          142    .rodata.gTIMER_0ClockConfig  ti_msp_dl_config.o
    0x000028d7   0x000028d7   0x00000001   PAD
    0x000028d8   0x000028d8   0x00000014   Data   RO          143    .rodata.gTIMER_0TimerConfig  ti_msp_dl_config.o
    0x000028ec   0x000028ec   0x00000002   Data   RO          144    .rodata.gUART_0ClockConfig  ti_msp_dl_config.o
    0x000028ee   0x000028ee   0x0000000a   Data   RO          145    .rodata.gUART_0Config  ti_msp_dl_config.o
    0x000028f8   0x000028f8   0x00000007   Data   RO           30    .rodata.str1.1      main.o
    0x000028ff   0x000028ff   0x00000001   PAD
    0x00002900   0x00002900   0x00000020   Data   RO          568    Region$$Table       anon$$obj.o


    Execution Region RW_IRAM2 (Exec base: 0x20000000, Load base: 0x00002920, Size: 0x00000e98, Max: 0x00001000, ABSOLUTE)

    Exec Addr    Load Addr    Size         Type   Attr      Idx    E Section Name        Object

    0x20000000   0x00002920   0x00000004   Data   RW          458    .data               mc_p.l(stdout.o)
    0x20000004   0x00002924   0x00000004   Data   RW          263    .data.K_V           l298n.o
    0x20000008   0x00002928   0x00000004   Data   RW          233    .data.Kd_Yaw        pid.o
    0x2000000c   0x0000292c   0x00000004   Data   RW          231    .data.Kp_Yaw        pid.o
    0x20000010   0x00002930   0x00000010   Data   RW           26    .data.black         main.o
    0x20000020   0x00002940   0x00000004   Data   RW          239    .data.max           pid.o
    0x20000024   0x00002944   0x00000002   Data   RW          266    .data.motorDuty_A   l298n.o
    0x20000026   0x00002946   0x00000002   Data   RW          268    .data.motorDuty_B   l298n.o
    0x20000028   0x00002948   0x00000010   Data   RW           25    .data.white         main.o
    0x20000038        -       0x00000050   Zero   RW          157    .bss.ADC_VALUE      adc.o
    0x20000088        -       0x00000004   Zero   RW           28    .bss.CalculateNormalizedValue.last_value  main.o
    0x2000008c        -       0x00000001   Zero   RW           32    .bss.Digtal         main.o
    0x2000008d   0x00002958   0x00000003   PAD
    0x20000090        -       0x00000004   Zero   RW          235    .bss.Err_Yaw        pid.o
    0x20000094        -       0x00000004   Zero   RW          234    .bss.Integral_Yaw   pid.o
    0x20000098        -       0x00000004   Zero   RW          232    .bss.Ki_Yaw         pid.o
    0x2000009c        -       0x00000004   Zero   RW          236    .bss.LastErr_Yaw    pid.o
    0x200000a0        -       0x00000010   Zero   RW           31    .bss.Normal         main.o
    0x200000b0        -       0x00000004   Zero   RW          237    .bss.Output_Yaw     pid.o
    0x200000b4        -       0x00000004   Zero   RW          273    .bss.SpeedL         l298n.o
    0x200000b8        -       0x00000004   Zero   RW          272    .bss.SpeedR         l298n.o
    0x200000bc        -       0x00000004   Zero   RW          264    .bss.Speed_Set      l298n.o
    0x200000c0        -       0x00000004   Zero   RW          265    .bss.Tarangle       l298n.o
    0x200000c4        -       0x00000004   Zero   RW          172    .bss.Tick           delay.o
    0x200000c8        -       0x00000004   Zero   RW          240    .bss.Yaw_Now_Correct  pid.o
    0x200000cc        -       0x00000001   Zero   RW          220    .bss.key_pressed    key.o
    0x200000cd        -       0x00000001   Zero   RW          221    .bss.key_start_pressed  key.o
    0x200000ce   0x00002958   0x00000002   PAD
    0x200000d0        -       0x00000004   Zero   RW          219    .bss.last_key_time  key.o
    0x200000d4        -       0x00000001   Zero   RW          267    .bss.pwmCounter_A   l298n.o
    0x200000d5        -       0x00000001   Zero   RW          269    .bss.pwmCounter_B   l298n.o
    0x200000d6   0x00002958   0x00000002   PAD
    0x200000d8        -       0x00000004   Zero   RW          270    .bss.pwmL           l298n.o
    0x200000dc        -       0x00000004   Zero   RW          271    .bss.pwmR           l298n.o
    0x200000e0        -       0x00000004   Zero   RW          238    .bss.result_angle   pid.o
    0x200000e4   0x00002958   0x00000004   PAD
    0x200000e8        -       0x000000b0   Zero   RW           29    .bss.sensor         main.o
    0x20000198        -       0x00000d00   Zero   RW           40    STACK               startup_mspm0l130x_uvision.o



  Load Region LR_BCR (Base: 0x41c00000, Size: 0x00000000, Max: 0x00000100, ABSOLUTE)

    Execution Region BCR_CONFIG (Exec base: 0x41c00000, Load base: 0x41c00000, Size: 0x00000000, Max: 0x00000080, ABSOLUTE)

    **** No section assigned to this execution region ****



  Load Region LR_BSL (Base: 0x41c00100, Size: 0x00000000, Max: 0x00000100, ABSOLUTE)

    Execution Region BSL_CONFIG (Exec base: 0x41c00100, Load base: 0x41c00100, Size: 0x00000000, Max: 0x00000080, ABSOLUTE)

    **** No section assigned to this execution region ****


==============================================================================

Image component sizes


      Code (inc. data)   RO Data    RW Data    ZI Data      Debug   Object Name

       112          0          0          0         80        831   adc.o
        90          4          0          0          4        962   delay.o
       148         16          0          0          6       4661   key.o
       872         68          0          8         26       4977   l298n.o
       736         96          7         32        197      10424   main.o
      1144          4          0          0          0       6720   no_mcu_ganv_grayscale_sensor.o
       256         40          0         12         28        882   pid.o
        20          4        192          0       3328        620   startup_mspm0l130x_uvision.o
      1842        168         67          0          0      29001   ti_msp_dl_config.o

    ----------------------------------------------------------------------
      5236        400        300         52       3680      59078   Object Totals
         0          0         32          0          0          0   (incl. Generated)
        16          0          2          0         11          0   (incl. Padding)

    ----------------------------------------------------------------------

      Code (inc. data)   RO Data    RW Data    ZI Data      Debug   Library Member Name

        64          8          0          0          0       4747   dl_adc12.o
        10          0          0          0          0        802   dl_common.o
        68          4          0          0          0       4504   dl_dma.o
       264        156          0          0          0      30121   dl_timer.o
        90          8          0          0          0      14127   dl_uart.o
         0          0          0          0          0          0   entry.o
         0          0          0          0          0          0   entry10a.o
         0          0          0          0          0          0   entry11a.o
         8          4          0          0          0          0   entry2.o
         4          0          0          0          0          0   entry5.o
         0          0          0          0          0          0   entry7b.o
         0          0          0          0          0          0   entry8b.o
         8          4          0          0          0          0   entry9a.o
        30          0          0          0          0          0   handlers.o
        80          6          0          0          0         72   idiv_div0.o
        48         10          0          0          0         68   init.o
         0          0          0          0          0          0   iusefp.o
        32          0          0          0          0         68   llshl.o
        38          0          0          0          0         68   llsshr.o
        34          0          0          0          0         68   llushr.o
        36          0          0          0          0         60   memcpya.o
        36          0          0          0          0        100   memseta.o
      2252         98          0          0          0        412   printfa.o
         0          0          0          4          0          0   stdout.o
        62          0          0          0          0         72   uidiv_div0.o
        96          0          0          0          0         84   uldiv.o
        40          2          0          0          0         68   cdrcmple.o
       356          4          0          0          0        140   dadd.o
        44          0          0          0          0         68   dcmple.o
       240          6          0          0          0         84   ddiv.o
       236          0          0          0          0        216   depilogue.o
        72         10          0          0          0         72   dfixi.o
        64         10          0          0          0         68   dfixul.o
        40          6          0          0          0         68   dflti.o
        28          4          0          0          0         68   dfltui.o
       208          6          0          0          0         88   dmul.o
       178          0          0          0          0        108   fadd.o
       130          0          0          0          0        144   fepilogue.o
        50          0          0          0          0         60   ffixi.o
        22          0          0          0          0         68   fflti.o

    ----------------------------------------------------------------------
      4992        350          0          4          0      56693   Library Totals
        24          4          0          0          0          0   (incl. Padding)

    ----------------------------------------------------------------------

      Code (inc. data)   RO Data    RW Data    ZI Data      Debug   Library Name

       496        176          0          0          0      54301   driverlib.a
      2764        122          0          4          0       1072   mc_p.l
      1708         48          0          0          0       1320   mf_p.l

    ----------------------------------------------------------------------
      4992        350          0          4          0      56693   Library Totals

    ----------------------------------------------------------------------

==============================================================================


      Code (inc. data)   RO Data    RW Data    ZI Data      Debug   

     10228        750        300         56       3680     114487   Grand Totals
     10228        750        300         56       3680     114487   ELF Image Totals
     10228        750        300         56          0          0   ROM Totals

==============================================================================

    Total RO  Size (Code + RO Data)                10528 (  10.28kB)
    Total RW  Size (RW Data + ZI Data)              3736 (   3.65kB)
    Total ROM Size (Code + RO Data + RW Data)      10584 (  10.34kB)

==============================================================================

